:10966100414952434F5445430056322E332D313236
:1096710021454E470042415454004241440040328A
:1096810044400040334440004F4646214E45574038
:109691004D454E55000A16000180000300007E0072
:1096A10000FE00001E0000360003E60001C40000B9
:1096B10000000FFFE053454152434840534154538A
:1096C1000043414C40414C54492020230056214144
:1096D1002152494F2020004241524F475220200041
:1096E100524F555445532020004E4541525354206A
:1096F10020005741595054532020004D21412152FF
:10970100214B2320200045584954213F002020208F
:1097110021415647212020202044535400214558FF
:1097210049540153454C40524F55544501534554FA
:109731002048454947485401464C4947485453201D
:109741006869015741595054532020686901524FAB
:1097510055544553202068690141495253504143B2
:109761004568690153455454494E4753686901019D
:10977100464C494748542D206869015245434F5290
:109781004445520153455454494E4753005345549F
:1097910020484549474854004750532048454947C8
:1097A1004854004241524F404845494748540047B8
:1097B100505320484549474854004C4F47424F4F6A
:1097C1004B20454D505459003E21455849540021E4
:1097D10045584954015245504C41590153454E4455
:1097E1000144454C45544500214558495401544EC6
:1097F100432031232035374B01544E432031232060
:10980100392E360101505743403130234035374B13
:1098110001505743403130234031394B01014D58FC
:1098210050403130234035374B014D5850203423BF
:109831002035374B014D58502031232035374B010E
:109841004D5850403130234031394B014D58502053
:1098510034232031394B014D5850203123203139E7
:109861004B002145584954014E4557202057415935
:1098710050540145444954205741595054014445DD
:109881004C202057415950540101434F4D3A015248
:109891004543454956452057500153454E442057AD
:1098A100415950540153454E4440414C4C4057504E
:1098B1000101444953542057502D57500144454C00
:1098C10040414C4C4057505400425247202144499A
:1098D10053540053544F52450050524553454E5432
:1098E10040504F532E005550444154494E472E2E5F
:1098F100004044454C4554454400574952450049B0
:10990100524441004C4953540053454E44002054A5
:1099110052414E534D4954204552524F522000213D
:10992100455849540153454C40524F555445014EF9
:109931004557202052544550540145444954205222
:109941004F555445015245564552534520525401F5
:1099510044454C202052544550540144454C20204C
:10996100524F5554450101434F4D3A01524543452C
:109971004956452052540153454E4420524F5554A7
:10998100450053454C21524F555445004E404540EA
:109991005700204E455740504F534021002140521F
:1099A10045564552534540005245565253002140B9
:1099B10044454C405750545300214044454C20529B
:1099C1005445004E4F5420454D50545920002140DC
:0D99D10053454E444052544500214558492D
:1099DE0054014C4F414420202043545201564945D6
:1099EE00572020204354520144454C40414C4C21B9
:1099FE0043545201434F4D3A015245435649564541
:109A0E00214354520153454E4420202043545200CA
:109A1E0056494557204354520020204D4F5645007D
:109A2E0020204D4F564520544F005343414C452066
:109A3E0020582F5920204558495400205343414C5B
:109A4E00450044495354204B4D0044495354204E35
:109A5E004D00214558495401564152494F2020206E
:109A6E0068690158432D53455420206869014745C4
:109A7E004E4552414C2068690101015445535446EC
:109A8E004C4947485401534552564943434F444568
:109A9E000142415349432D53455401454153592DDC
:109AAE0053455400544553545300214558495401CD
:109ABE0053494E4B212D0153494E4B404D4F4401BE
:109ACE0053494E4B40494E560154454320202040A9
:109ADE00303040250156415220544340202040232F
:109AEE0001564F4C554D4501564152494F204E554A
:109AFE004C4C004E4F542150524553454E54005637
:109B0E004152494F204E554C4C004B45455040510B
:109B1E0055494554403130404D494E004245464F1F
:109B2E005245204E554C4C494E47002145584954FC
:109B3E00014155544F43454E54014156472F444918
:109B4E00535401474C444550415448014C402F401A
:109B5E0044202020202E01534C494E450143594CA0
:109B6E00530143594C01545241434B00214558492E
:109B7E00540101554E495401434C49434B40302C3E
:109B8E0040202301434F4E5452415354014E4D45F4
:109B9E0041213138330040574159504F494E5420DE
:109BAE004558495354534000574159504F494E540C
:109BBE000020204558495420202100524543454954
:109BCE005645004652454540004C4F4144494E478C
:109BDE002E0053455256494345005341543A004FC7
:109BEE00464620202020202020200047505320458C
:109BFE0052524F520053544F52494E472E2E00523E
:109C0E004F555445004E454152455354004C49530F
:109C1E0054200045544500414C54403000454D50B1
:109C2E00545920525445200020544F4F404D554317
:109C3E00482000214053454C404C4953540020537A
:109C4E00454C405750544021002140524543454910
:109C5E00564540002020404F204B40202021004FF1
:109C6E004B0020204641494C202021004641494CC2
:109C7E000020455849540045444954005940454038
:109C8E0053004544495420204E4557202053544FED
:109C9E005245005843542D464C49474854200055D0
:109CAE0053454400454E54455220004D4D2E4D4DCA
:109CBE004D20004D4D2753532E53005747532138F7
:109CCE0034002040554054404D40200055405440F3
:109CDE004D002055544320005357495353474400D9
:109CEE00414C5400535549405800415647003530B9
:109CFE0030003136343000205D203130404B632F40
:109D0E0070005D2020203140632F2300205D202035
:109D1E0035404B5453005D203230304046504D009C
:109D2E00404947432056414C494400494743405718
:109D3E00414954202023004947432D4C4F47474566
:0D9D4E00520020532F4E3B00205345414C46
:109D5B0045442000554E5345414C45440048572D32
:109D6B005645523B40202C0046572D5645523B4002
:109D7B00202C00205348454C4C200040434F4E4E66
:109D8B0045435420200031313532303000205540CE
:109D9B00534042200054494D454F555440004C4FC1
:109DAB0043414C00214558495401474C49444552C5
:109DBB0053206869015441534B532020206869019B
:109DCB0053455455502020206869012D2D2D2D2DE4
:109DDB002D2D2D2D2D014B2D454E4C012020454E6B
:109DEB004C3D0147464143404B4559015345544077
:109DFB00495341404D534C0144554D5040464C4105
:109E0B00534801434C522040464C41534800544563
:109E1B004D504C4154450050494C4F543A00474C1F
:109E2B004944455220545950453A00474C49444502
:109E3B00522049443A00434F4D502E49443A004377
:109E4B004F4D502E434C4153533A002145584954E2
:109E5B000152442D45450152442D464C4153480176
:109E6B00474838300144454C20414C4C20464C006F
:109E7B002145584954015241444955534020202112
:109E8B002201494E54562049402020212301494E9E
:109E9B005456414C4020202123015452542F4753F8
:109EAB005000406340204B63004654204B630040FE
:109EBB006340204E4D004654204E4D003022003062
:109ECB0066004D2F53003230305E003530305E006F
:109EDB003122003222003322003522003822004684
:109EEB004C3700464C313600464C333300464C362B
:109EFB003500463130300046313630004632363090
:109F0B00005E252640534F47005E252640544153A3
:109F1B0000414C540056415200225E2F24004B54FA
:109F2B005300532F4E002224004B5400225E004E50
:109F3B004D00302C3500312C3000322C3000302CC1
:109F4B003600312C3200322C3500332C3800372CB4
:109F5B00350040313500403330004036300020545E
:109F6B005241434B214F4E20200020545241434B32
:109F7B00214F464620003C2D204C495354202D3E6A
:109F8B002020455849540053454C004E4558540029
:109F9B005441534B00464C2D444154450054500002
:109FAB00544F46005354410046494E004C414E001D
:109FBB00534554204F46465345540049534120487E
:0E9FCB00454947485400424C4120424C410059
:1051EA0030482475A7049005C2E0F51CE0F51DE0DF
:1051FA00F51EE0F51FE0F56DE0F56EE0F56FE0F500
:10520A0054125DAA1257EA2275C70375C6E475B926
:10521A0001E5BCB48143125DAA1267DC8E628F631A
:10522A007568F97569001252C0203C2D203B2B127B
:10523A0053F51253C9856D1C856E1D856F1E8554E5
:10524A001F12532C203C12203243201D231253F5E7
:10525A001257EAE532242850DC2212532C203CF95A
:10526A00203DF6203205201DBD80EF301DB880EAB2
:10527A001253F51257EA856D1C856E1D856F1E85C2
:10528A00541F1253DF1257EA203DCE809912561846
:10529A00201D0D755310740012557B203DBB80866E
:1052AA00E553540FC553C4540F203505125490804A
:1052BA000312557B808BC23CD23B12537CFD1253A6
:1052CA007CFC12537CC39573F565EC9574F564ED1B
:1052DA009575600504600A800EE56424E05011802B
:1052EA0006E5642420400912537C12537C02537C45
:1052FA0012537CFD12537CFC12537CC39576F567DE
:10530A00EC9577F566ED9578600904600122E5660B
:10531A00F48002E5668562F0A474E025F04002C2DA
:0D532A003B22C23C12537CA2E7923DA2E65A
:10533700921DA2E592324026A2E492E592E692E718
:10534700FC12537C2565F565EC3564F56412537CD6
:10535700FC12537C2567F567EC3566F56622A2E4F7
:105367009235540F79C6F712537C09F7301D051291
:10537700537CF55322E5697023E5686030240240C9
:105387002C24FE75F004A485F0C7F5C675B901E5B0
:10539700BCB4811985BD68756902801E54037010FD
:1053A70005C675B901E5BC056953690F22D23C22D0
:1053B700147004E5BD80F0147004E5BE80E9E5BF14
:1053C70080E575A7009006F6E56DF0A3E56EF0A3FE
:1053D700E56FF0A3E554F02275A7009006F6E0F517
:1053E7006DA3E0F56EA3E0F56FA3E0F55422E56445
:1053F700B2E7F56D85656EAB67E566FC30E707C319
:10540700E49BFBE49CFCAA62A9631264F6E56630A0
:10541700E707C3E49DFDE49EFEEEB2E7F56F8D540A
:105427002275380C1256811256CCD5530122753885
:105437000C1256521256C2D5530122753800125615
:0E5447006A125691D553012275380012565242
:10545500125691D55301227538031256811256FD05
:10546500D55301227538031256521256F3D55301FE
:105475002275380F12566A125722D55301227538F4
:105485000F125652125722D5532622905495237344
:105495008091807780688059804A803B802C801D70
:1054A500800E80DA80CB80BC80AD809E808F80802E
:1054B500753815125681125744D553012275381582
:1054C500125652125739D553012275380912566AA8
:1054D50012570AD553012275380912565212570A26
:1054E500D55301227538061256811256B4D553018B
:1054F500227538061256521256A9D553012275380F
:105505001212566A1256DAD55301227538121256FE
:10551500521256DAD55301220254287538151256FF
:1055250081125744D553012275380F12565212571E
:1055350022D553012275380F12566A125722D553B8
:1055450001227538031256521256F3D553012275AE
:1055550038031256811256FDD553012275380012B3
:105565005652125691D553012275380012566A12B9
:105575005691D55326229055802373809E80A9800D
:10558500B480BF80CA80D580E08010801B802680D3
:1055950031803C80478052805D806875380C12569A
:1055A500521256C2D553012275380C125681125625
:0E55B500CCD55301227538121256521256DA16
:1055C300D553012275381212566A1256DAD5530191
:1055D300227538061256521256A9D5530122753830
:1055E300061256811256B4D5530122753809125644
:1055F3005212570AD553012275380912566A1257A7
:105603000AD5530122753815125652125739D553FC
:10561300012202552078C686040886037AED1264B7
:10562300B478CAA60408A60378C686040886037A53
:10563300621264B478CCA60408A60378C68604086C
:1056430086037AB51264B478C8A60408A603227543
:105653001A6A751B0A78CA8618088619125893782D
:10566300CC86060886072278C88618088619E4F5CA
:105673001AF51B12589378C886060886072278C63F
:105683008618088619751A00751B01025893E51DC3
:105693002519F51DE51C3518F51CC3E51F9FF51FDE
:1056A300E51E9EF51E22C3E51F9FF51FE51E9EF511
:1056B3001EC3E51D9519F51DE51C9518F51C22E57E
:1056C3001D2FF51DE51C3EF51CC3E51F9519F51FA0
:1056D300E51E9518F51E22C3E51D9FF51DE51C9ECD
:0956E300F51CC3E51F9519F51F24
:1056EC00E51E9518F51E22E51F2FF51FE51E3EF54C
:1056FC001EE51D2519F51DE51C3518F51C22C3E505
:10570C001D9519F51DE51C9518F51CE51F2FF51FAA
:10571C00E51E3EF51E22E51D2FF51DE51C3EF51C74
:10572C00E51F2519F51FE51E3518F51E22C3E51DCD
:10573C009FF51DE51C9EF51CE51F2519F51FE51EA3
:10574C003518F51E22E51A7009E51B70058C068DBF
:10575C000722ED851BF0A4A2F792D5ED851AF0A4D3
:10576C00AEF0FFEC851BF0A4A2D53FEE35F0FF9216
:10577C00D5EC851AF0A42FFFE435F030D50104FEEA
:10578C0022E4F51AF51BEF4E7003051B22EF651989
:10579C007006EE65187001227808C3EF33FFEE3304
:1057AC00FEEF9519F5F0EE95184003FEAFF0E51AF3
:1057BC0033F51AD8E5F4F51A751BFF7805C3EF33EA
:1057CC00FFEE33FEEF9519F5F0EE95184003FEAFA2
:0357DC00F0E51BDA
:1057DF0033F51BD8E5F4C403F51B22E51D9511E540
:1057EF001C9510500BE56E9511E56D95105001222B
:1057FF00E51F9511E51E9510500BE5549511E56FBA
:10580F009510500122E51D9513E51C9512400BE5EF
:10581F006E9513E56D9512400122E51F9513E51E58
:10582F009512400BE5549513E56F951240012275C3
:10583F002C00C3E51F9554FFE51E956FFE92605037
:10584F0007C3E49FFFE49EFEC3E56E951DF519E5C2
:10585F006D951CF5189261500BC3E49519F519E479
:10586F009518F518C3E5199FE5189E9262500AE541
:10587F0018CEF518E519CFF51912578DE52C75F0DF
:10588F0003A4F538E538905899730258B10258C5FA
:10589F000258D30258EB0258FE02591102591F0247
:1058AF005937851C16851D17C3E4951FF515E4950B
:1058BF001EF51402594A851C16851D17851E148561
:1058CF001F158077C3E4951DF517E4951CF516C3D6
:1058DF00E4951FF515E4951EF514805FC3E4951D3F
:0558EF00F517E4951C13
:1058F400F516851E14851F15804CC3E4951FF517F6
:10590400E4951EF516851C14851D158039851E1613
:10591400851F17851C14851D15802BC3E4951FF561
:1059240017E4951EF516C3E4951DF515E4951CF5CD
:10593400148013851E16851F17C3E4951DF515E401
:10594400951CF5148000C3E5179513E51695121000
:10595400D70122E5159513E514951210D70122E518
:1059640019F92517FFE518F83516FED3EF9511EE52
:105974009510500122E5119517FDE5109516FC4090
:105984002A4D6027125751E5152FF515E5143EF5FC
:1059940014E5159513E514951210D70122E5199D08
:1059A400F9E5189CF8851016851117E51729FFE508
:1059B4001638FEE5139FE5129E500BC3E5139517A9
:1059C400F9E5129516F8E51A700AE51B7006AA00A7
:1059D400AB018013E9851AF0A4E5F0FBE8851AF021
:1059E400A42BFBE435F0FAE5152BFBE5143AFAE5B4
:0559F400119BE5109A73
:1059F90010D70122EB9515FDEA9514FCC3E5159521
:105A090011E514951010D717E5139BE5129A503636
:105A1900E5139515FFE5129514FE125CC78027EB77
:105A29009511FFEA9510FEAA00C001125CC7D003C8
:105A3900E5172BFBE5163AFAEB99F517EA98F516EF
:105A4900851115851014C2D5E5466002D2D5AA562E
:105A5900E98AF0A4ABF0E88AF0A42B30D50475F0FC
:105A69000384F8700122E5172513FDE5163512FCAC
:105A7900ED8AF0A4ABF0EC8AF0A42B30D50475F0D4
:105A89000384FEE5152513FDE5143512FCED8AF0B6
:105A9900A4ABF0EC8AF0A42B30D50475F00384F99B
:105AA900E538905AAF73025AC7025AD3025ADC0238
:105AB9005AE5025AEB025AF7025AFE025B03C37413
:105AC9003E9EFFC3743E99FE8032C3743E9EFFAE74
:105AD900018029AF06C3743E99FE8020AF06AE014E
:0E5AE900801AC3743E9EFEC3743E99FF800E69
:105AF700C3743E99FF8007C3743E9EFEAF0108EF53
:105B07002437FFE51B7007E51A700CE8800EA2E743
:105B1700E51A50030460F488F0A4E5F0600104F985
:105B270023FA98FBC3E998C333F9905B37E53873D9
:105B3700025B4F025B7C025BB1025BDE025C0B0225
:105B47005C38025C65025C9205A7800BEB30E703CB
:105B57002A8002291E1FFBEEC45403F583EE540866
:105B6700C42FF582EE5407243883F5F0E045F0F0B2
:105B7700D8DA05A72205A7800BEB30E7032A8002B6
:105B8700290E1FFBEEC45403F583EE5408C42FF50A
:105B970082EE5407240B83F5F0E045F0F0D8DA05E0
:105BA700A722804020100804020105A7800BEB30D4
:105BB700E7032A8002291E0FFBEEC45403F583EE88
:105BC7005408C42FF582EE540724EC83F5F0E04522
:105BD700F0F0D8DA05A72205A7800BEB30E7032AF8
:045BE7008002290E01
:105BEB000FFBEEC45403F583EE5408C42FF582EE7D
:105BFB00540724BF83F5F0E045F0F0D8DA05A7226F
:105C0B0005A7800BEB30E7032A8002291F1EFBEE52
:105C1B00C45403F583EE5408C42FF582EE540724C5
:105C2B009283F5F0E045F0F0D8DA05A72205A780BE
:105C3B000BEB30E7032A8002291F0EFBEEC4540343
:105C4B00F583EE5408C42FF582EE5407246583F5D3
:105C5B00F0E045F0F0D8DA05A72205A7800BEB3072
:105C6B00E7032A8002290F1EFBEEC45403F583EED3
:105C7B005408C42FF582EE5407243883F5F0E04521
:105C8B00F0F0D8DA05A72205A7800BEB30E7032A43
:105C9B008002290F0EFBEEC45403F583EE5408C4A7
:105CAB002FF582EE5407240B83F5F0E045F0F0D886
:105CBB00DA05A7228040201008040201EC701FEDCA
:085CCB0020E740D2E023CF23C3
:105CD300CF30E7F980357B08801A7B1080167B2054
:105CE30080127B40800E20E4ED20E3EE20E2EF20E3
:105CF300E1F07B80EE8BF0A4CF8BF0A4E5F02FFFD7
:105D0300EC8BF0A4CD8BF0A4E5F02D2499838FF0D8
:105D1300A433E5F033FBE98BF0A4E5F0C88BF0A4E2
:105D230028F9E435F0F822FFFEFCFAF8F6F4F2F075
:105D3300EFEDEBEAE8E6E5E3E1E0DEDDDBDAD9D738
:105D4300D6D4D3D2D0CFCECCCBCAC9C7C6C5C4C391
:105D5300C1C0BFBEBDBCBBBAB9B8B7B6B5B4B3B2A8
:105D6300B1B0AFAEADACABAAA9A8A8A7A6A5A4A392
:105D7300A3A2A1A09F9F9E9D9C9C9B9A9999989753
:105D830097969594949392929190908F8F8E8D8DF8
:105D93008C8C8B8A8A898988878786868585848483
:105DA3008383828281818075A700905DD0E546FA66
:105DB30024FA50027A05EA2323F978107F0493F634
:105DC3000809E9DFF9905DE8EA93F556227FC2807E
:105DD3003E7F4680BA7E8C81747D1882E87A308556
:105DE300D074608BA0808040201008125DF40260A4
:105DF30048D215D234D274D273C219C23A1267DCB4
:105E03008E47757D007546057552021295FE120880
:105E130054E53524E250031295FEE55275F016A4BD
:105E2300F570125FFE755115125EC27F237E0990D5
:105E33009A2712731812D30F10000810010D1002C5
:105E43001280E2125F7175330180DA125FB6753327
:105E53000180D2755100125EC27E00909A3812738F
:105E63004B7F237E05909A2E127318125F1A12D35A
:105E73000FE55210000F10010510029280D5045453
:105E830003F55280CE125EC27F237E0B909A491295
:0D5E93007318E5466007146004141243FD07
:105EA00012D30FE54610000810010B10021180D824
:105EB00060D6154680D2B4050280CD054680C90261
:105EC0005E1175320012D4C37F017E11909A1E12AA
:105ED000734B7F2F7E0090CCDC12CA047E3C90CCAA
:105EE000DC12CA04E55112CC7B75170812CE6A1277
:105EF000442D75710012CF12741BFFF5177E0F90A1
:105F00009A50305D03909A5812734B129641126D5D
:105F100018124805125212022252E55260141460FF
:105F20001E1460297F647E2D791C125F641E1FD9A8
:105F3000F9227F6A7E1F7928125F641FD9FA227FB7
:105F4000487E2D791C125F640F1ED9F9227F567E80
:105F50003379281F12D4060F0F12D4061F12D4064D
:105F60001ED9F0221E12D4060E0E12D4061E02D422
:105F700006E552605514606814606D800075709E6F
:105F8000125FEB8003757000E5732540F573E4350F
:105F900074F574E43575F57522757016125F888096
:105FA0000375702DE5762542F576E5773541F57771
:105FB000E43578F57822E55260CB1460DC1460E1BA
:105FC0008000757044125FA4800375705AE5739564
:0D5FD00040F573E5749400F574E5759400D8
:105FDD00F57522757071125FCD8003757088E57649
:105FED009542F576E5779541F577E5789400F57866
:105FFD0022E54690601493F540FEAD47E4FFFC1298
:10600D0065898E418F4222020C183060C07F371295
:10601D00170912226812D30F1262F6EB70059097D2
:10602D00C2800B1260D5909C625003909C707F369D
:10603D007E0412731812D30F12D3DAE4F535F5205E
:10604D007537099099DA12215690605A73020946F4
:10605D00026222025DEE02632702606F0260880217
:10606D00601A7F25121A8180D27F2D7E04909C3676
:10607D0012731812D30F12D3DA80C07F2E121709A4
:10608D0012226812D30F1262DA124987D2AC1000B5
:10609D00AA306DFA126185203BCF40ED7568F97518
:1060AD0016001261D540FB1263947F2E7E35E516E6
:1060BD0012C94212D30F05161273BE78C6B6F7E297
:1060CD001263437F2D0262C97C0312498712D0A54A
:1060DD00744112D0D8745312D073EB12D094127342
:1060ED00D05003DCE5227515F975160010000EE58C
:1060FD00156025126127400512614E5002D3227F93
:10610D00367E29E51612C88B12D30F7F1412D3EDEC
:10611D000516E51664F870D4C32212794975B901D4
:10612D00E5BCB4811AE5BDF51570037516F778C693
:08613D00A616127A92127A8A6A
:10614500127A8AC3027A8AD3227F0375F019D5E0C1
:10615500FDD5F0FA12498712D0A5744112D0D87432
:106165004212D0737E0F78C6E60812D073DEF9129C
:10617500D0971273D0400122DF012275F00080CE46
:10618500C23B124987D2AC12D219C5F0603EC5F0A8
:10619500B440F412D21EB4400312D21EB4412DF500
:1061A5003812D21EB4532512D21EFA12D21EE53869
:1061B500701A12D21EB40D1412D21EB40A0EC3E503
:1061C500169A40030273B5C2ACD23B22C2ACD322AD
:1061D500127413124987D2AC1000F112D219C5F00E
:1061E50060EAC5F0B440F112D21EB4400312D21ECB
:1061F500B441D9F53812D21EB442D17E1078C612F8
:10620500D21EF608DEF9E53870C212D21EB40DBCF6
:1062150012D21EB40AB6C2ACC3220260487F0A126B
:10622500170912226812D30F1262DA1249D9D2ACB9
:106235001000E712D21EB440F5F53812D21EB46E26
:10624500ED12D21EE538600A1249D9744F12D07F7B
:1062550080DC7F0A7E35E51612C94212D30F12D0B3
:10626500D3E51612D07F12D0897568F9751600121C
:1062750049D9D2AC10005B12D21EB440F7F53812E2
:10628500D21EB44EB97E1078C612D21EF608DEF9BB
:106295001249D9E5386007744F12D07F80D1126357
:0562A500940516745180
:1062AA0012D07F78C6B6F7C212634312D3E17F0ACF
:1062BA007E35E51612C94212D30F12D3E17F097E49
:1062CA0035909C6D12731812D30F12D3DD026048F9
:1062DA0075150075160512794075B901E5BC30E7E8
:1062EA000205160515E515242050EB227B007515CD
:1062FA00F912794975B901E5BCB481010B0515E5B7
:10630A0015240250EC75150112794075B901E5BCE6
:10631A00B481010B0515E515242050EC227F1C12CF
:10632A0017091222AB12D30F10000B10010280F8CA
:10633A007515F9126343026048E515603724024077
:10634A001A241E5019E5152407400280271279499C
:10635A0012637F0515E515240250F27515011279AD
:10636A004075B901E5BC30E70312637F0515E515F1
:10637A00242050EA2212B416124F9805C6124F98DA
:10638A0005C6124F9805C6024F98E568606AF5156A
:10639A000515E5152402501D75150112794075B9C8
:1063AA0001E5BC30E70280190515E515242050EBFC
:1063BA00751500800C241E60F750E0E51524065080
:1063CA0037E56875F004A485F0C7F5C675BC81E5A4
:1063DA0015F5BDF56878C6B6F70375BD00081263F2
:1063EA00F71263F11263F186BC0886BD0886BE08FF
:0963FA0086BF08124F9805C62267
:10B86C0012A79F12B96B127E5C12B8F0127E641292
:10B87C00B8FD02A7A312A79F12B96B127E5C7F5A68
:10B88C00C23C127D3E127F3A783F79437F607EEA5C
:10B89C0012B95F127E647F65127D3E127F3A783D4D
:10B8AC0079417F207E4E12B95F303C2012BB2112B1
:10B8BC00B97C783F794312B8DB783D794112B8DB1B
:10B8CC0012BB2178D7E65480F67537000282B6C3D6
:10B8DC00E796FF1819E796FE0809C3E69FF71819B3
:10B8EC00E69EF7227F5B7E06909CF212734B1F80C4
:10B8FC000A7F667E14745912C9A41F127BC77E3945
:10B90C00E402C9C37866E620E73418C3E6947208EB
:10B91C00E694045029C318E6941F08E69404401ECC
:10B92C007869E620E71818C3E6940E08E6940150EF
:10B93C000DC318E6947508E694004002D322C32286
:10B94C00E67D0030E7011D08E62BFB18E63CFCE425
:0EB95C003DFD22C3EB9FF6F71819EC9EF6F79F
:10B96A002212B910400CE47842F608F67840F6083C
:10B97A00F6227864C3E6946AF55708E6944CF556BD
:10B98A000808C3E69458F55B08E694AEF55A75398B
:10B99A0000AC56AD57EC12AB4C784C12ABDAAC5A41
:10B9AA00AD5BEC12AB4C785012ABDA7F2B7E867D06
:10B9BA00777C1812AB11785012ABCE12AA1D12ABBB
:10B9CA0011785012ABCE12AA1D12AB11785012ABDD
:10B9DA00CE12AA1D12AB117F367E847D257C64129D
:10B9EA00AB11785012ABCE12AA1D12AB11784C12C1
:10B9FA00ABCE12AA1D12AB117F3F7EA27D607C8B5B
:10BA0A0012AB11785012ABCE12AA1D12A80B12A8B3
:10BA1A000B12ABE67F3F7E807D057CE6053912AAD4
:10BA2A001D784812ABDA7F2C7E937D477C7F12AB60
:10BA3A0011785012ABCE12AA1D12AB11785012AB6C
:10BA4A00CE12AA1D12AB11784C12ABCE12AA1D123D
:10BA5A00AB117F357EB47DF87CDF12AB11785012C2
:10BA6A00ABCE12AA1D12AB11785012ABCE12AA1D80
:10BA7A0012AB117F3F7EED7D227CCD12AB11784C4B
:10BA8A0012ABCE12AA1D12A80F12A80B784412AB41
:10BA9A00DA7F317E397D9D7CE712AB11784C12AB8F
:10BAAA00CE12AA1D12AB11784C12ABCE12AA1D12DD
:04BABA00AB11784410
:10BABE0012ABCE12A80F12AB117F2C7E377D0C7CF1
:10BACE00A312AB11784C12ABCE12AA1D12AB117889
:10BADE004C12ABCE12AA1D12AB11784C12ABCE1279
:10BAEE00AA1D12A80F12ABE67F3F7E807D027C9FBF
:10BAFE00053912AA1D784412ABDA784812ABCE1271
:10BB0E00AB838E428F43784412ABCE12AB838E4002
:10BB1E008F4122753900AC42AD43EC12AB4C7848E4
:10BB2E0012ABDAAC40AD41EC12AB4C784412ABDA4E
:10BB3E007F2B7E537D507C0912AB11784812ABCE11
:10BB4E0012AA1D12AB11784812ABCE12AA1D12AB5F
:10BB5E0011784412ABCE12AA1D12AB117F347EF2B5
:10BB6E007DCD7CA312AB11784812ABCE12AA1D125A
:10BB7E00AB11784812ABCE12AA1D12AB117F3F7ECD
:10BB8E000A7D2E7CAE12AB11784412ABCE12AA1DDA
:10BB9E0012A80B12A80B784C12ABDA7F2B7E4F7DBE
:10BBAE00AF7CB212AB11784812ABCE12AA1D12ABFB
:10BBBE0011784812ABCE12AA1D12AB11784812ABF7
:10BBCE00CE12AA1D12AB117F357EB17D4B7C951224
:10BBDE00AB11784812ABCE12AA1D12AB11784412DB
:10BBEE00ABCE12AA1D12AB117F3F7E497DCD7C4597
:10BBFE0012AB11784812ABCE12AA1D12A80F12A8C2
:10BC0E000B785012ABDA784C12ABCE12AB838D554B
:10BC1E008E568F57785012ABCE12AB838D598E5AEB
:04BC2E008F5B78644C
:10BC3200E557246AF608E556344CF608E55534040F
:10BC4200F608E55B2458F608E55A34AEF608E43502
:03BC520059F6227E
:1081040012A79F12879512A7A37F66909CDA127319
:10811400491281727F5A78C412814E12815678C6F0
:1081240012814E1281397F6578C812814E128156B0
:1081340078CA12814E7E2DE51B12C9C37E33E51A1F
:1081440012C9C37E39E51902C9C38604088603022D
:1081540064537E15E51C12C9C37E1BE51B12C9C3FB
:108164007E21E51A12C9C37E27E51902C9C37F5AC5
:108174007E01E53A12C8D97E0B908B89E53B9302C8
:10818400C9D6E6FF08E6FE08E6FD339217E450017F
:10819400F4FC12ABF775130A75390112ADF578D7F3
:1081A400E6C2E775F00A84F9303D02A9F012ABF794
:1081B4008913053912ADCE30170A053912ADE10520
:1081C4003912ADE1A80302ABDA12A79F128795C258
:1081D4003C7F5A7E031280EB12817212D30F10007F
:1081E4000810011510022080EFE53A146004153AD6
:1081F4008003753A3CD23C80DFE53AB43C05753ADD
:108204000180F2053A80EE7E031280E67E0B128036
:10821400EB12817212D30F10000810011510022006
:1082240080EFE53BB40205753B158002153BD23C5B
:1082340080DFE53BB41505753B0280F2053B80EE1B
:108244007E0B1280E67F5A78C412814E1281561238
:0782540082BF127F4A78C4CB
:10825B0012831778C612814E1281391282F1751C66
:10826B0000127F4A78C61283177F6578C812814E39
:10827B001281561282BF127F4A78C812831778CAAE
:10828B0012814E1281391282F1751C00127F4A78CD
:10829B00CA128317303C14E53B24F4500B78C9E623
:1082AB002410F618E63427F612831D12A7A3127AB0
:1082BB00CC02D30FC2247E15E51C12803BF51CD2D9
:1082CB00247E1BE51B12803BF51B1023E77E21E56B
:1082DB001A12803BF51A1023E67E27E51912803B14
:1082EB00F5191023E822C2247E2DE51B12803BF5E5
:1082FB001BD2247E33E51A12803BF51A1023E77E3E
:10830B0039E51912803BF5191023E622ECF608EB40
:10831B00F622128BA178C8E6FE0886073395E0FD9E
:10832B00FC12AB117FE87E037D007C0012ADF512D1
:10833B00AB1178CAE6FE0886073395E0FDFC12AD5B
:10834B00CE12AB117F807E697D677CFF12ADCEECC8
:10835B0012AB4812AB117F3F7E807D0D7C1D12AAA4
:10836B001D12AB117F3D7E407D007C0012AB11785E
:10837B00BC12ABCE12AA1D12AB117F3E7E807D00CC
:10838B007C0012A80F12AB1178BC12ABCE12AA1D37
:09839B0012AB117F3F7E807D00D2
:1083A4007C0012A80B12AB1178B412ABCE12AA1D2A
:1083B40012AA95783C12ABDA7F407E807D007C0067
:1083C40012AB11783C12ABCE12AA1D12AC7412ABD4
:1083D400117F3F7EA87D007C0012AB1178B812ABF0
:1083E400CE12AA1D12AA1D12AB117F407E007D0081
:1083F4007C0012AB11783C12ABCE12AA1D12AC74E5
:1084040012AB117F3F7EC07D007C0012AA1D12A812
:108414000F12AB1178B812ABCE12AA1D12AB1178A1
:108424003C12ABCE12A80F785412ABDA12AC5E78C1
:108434005812ABDA12AB1112AA1D12AB1178C0128A
:10844400ABCE12AA1D784412ABDA785412ABCE121A
:10845400AC74783C12ABDA12AB1112AA1D12AB1138
:1084640078BC12ABCE12AA1D783C12ABDA7F3E7EEA
:10847400C07D007C0012AB11783C12ABCE12AA1D59
:1084840012AB117F3F7E007D007C0012A80F12AB5F
:1084940011783C12ABCE12AA1D12AB117F3F7E8025
:1084A4007D007C0012A80F12AB1178B412ABCE126F
:1084B400AA1D787012ABDA78C4E6FE0886073395F5
:1084C400E0FDFC12AB117FE87E037D007C0012AD61
:1084D400F512AB1178C6E6FE0886073395E0FDFC7D
:1084E40012ADCE12AB117FE07E5E7DF87CFF12AD43
:1084F400CEEC12AB4812AB117F3F7E7F7DE57CC989
:0585040012AB117870BC
:1085090012ABCE12AA1D12AA95785012ABDA7F3F90
:108519007EF07D007C0012AB11783C12ABCE12AA22
:108529001D12AB117F3F7EC07D007C0012A80F1287
:10853900AB11783C12ABCE12AA1D12AB117F3F7E54
:10854900807D007C0012A80F783C12ABDA78BC124F
:10855900ABCE12AB117F3F7E807D007C0012A80B51
:1085690012AB11783C12ABCE12AB1178B412ABCE70
:1085790012AA1D12AA1D784012ABDA785412ABCE9A
:1085890012ACAC783C12ABDA12AB1112AA1D78749A
:1085990012ABDA7F417E107D007C0012AB1178C0EE
:1085A90012ABCE12AA1D12AB117F407E807D007CDA
:1085B9000012AB11784412ABCE12AA1D12AB117F77
:1085C900417E207D007C0012A80B12AB1178441269
:1085D900ABCE12AA1D12AB117F407E407D007C00FC
:1085E90012AB11787412ABCE12AA1D12AB117F40D7
:1085F9007EA07D007C0012A80F12A80F12A80B12F2
:10860900AB11785012ABCE12AA1D12AB11785012D1
:10861900ABCE12AA1D12AB117F3D7E2A7DAA7CAB7F
:1086290012AA1D12AB117F3F7E007D007C0012A8AB
:108639000B12AB11783C12ABCE12AB11787012ABA6
:10864900CE12AA1D12AB11784012ABCE12AA951206
:10865900AB11785012ABCE12AA1D12AB1178501281
:10866900ABCE12AA1D12AA1D12AB11785412ABCEB1
:0C86790012A80B12AB117F4A7E517DD27B
:108685007CCB12AA1D12AB8378AC12ABDA7F407E8D
:10869500007D007C0012AB11787412ABCE12AA1DBE
:1086A50012AB117F3F7E807D007C0012A80F12ABBC
:1086B50011784412ABCE12A80F12AB11785012AB41
:1086C500CE12AA1D12AB11785012ABCE12AA1D12F2
:1086D500AB11785012ABCE12AA1D12AB117F3E7EA4
:1086E5002A7DAA7CAB12AA1D12AB11785012ABCE13
:1086F50012A80B12AB11785812ABCE12AA9512AB79
:10870500117F4A7E517DD27CCB12AA1D12AB8312FA
:10871500AB11AF3AEF3395E0FEFDFC12AB117F4094
:108725007E7E7D057C0012ADF512AB117F607E75F6
:108735007D587CFF12ADCE12ADCE78B012ABDA7893
:10874500AC751B6412876C8F1C78B0751B6712871C
:108755006CE51C75F00AA42FFF249C50027F00785D
:10876500D7E654802FF62275390012ABCE12AB1125
:108775007F0A7E007D007C0012AEA1A81BE513F6E2
:1087850008E512F608E511F6335004EFF404FF226C
:10879500C23D78647BAC128186D23D78677BB0128E
:1087A5008186128BA17F007EE47D577C0012AB1180
:1087B50078AC12ABCE12ADCE12AB117F007E537DDD
:0E87C500077C0012AEA112AB3085133B7F8003
:1087D3007ECB7DA47C0012AB1178B012ABCE12AD70
:1087E300CE12AB117F407E7E7D057C0012AEA112BE
:1087F300AB30E513F56F04F53A85126E85116D857F
:10880300106C7F407E7E7D057C0012AB11786C126C
:10881300ABCE12ADF512AB117F607E0C7DA27C0056
:1088230012AB1178B012ABCE12ADCE12ADE1786CB3
:1088330012ABDA78AC12ABCEEC12AB4812AB117FB1
:10884300347E9C7D2B7C5F12AA1D785412ABDA1206
:10885300AC5E785012ABDA786C12ABCEEC12AB484C
:1088630012AB117F347E9C7D2B7C5F12AA1D12AB51
:1088730011785012ABCE12AA1D784012ABDA7F40AA
:108883007E007D007C0012AB11785412ABCE12AA8D
:108893001D12AC7412AB117F3D7EC07D007C0012B3
:1088A300AB1178BC12ABCE12AA1D12AB117F3E7E68
:1088B300C07D007C0012A80F12AB1178BC12ABCEA6
:1088C30012AA1D12AA1D12AB117F3D7E407D007CB2
:1088D3000012AB1178BC12ABCE12AA1D12AB117FE2
:1088E3003E7E807D007C0012A80F12AB1178BC1273
:1088F300ABCE12AA1D12AB117F3F7E807D007C00A0
:1089030012A80B12AB11785412ABCE12AA1D12A8E7
:108913000B12AB117F407E807D007C0012AB11787F
:108923005412ABCE12AA1D12AC7412AB117F3D7E52
:10893300707D007C0012AB1178BC12ABCE12AA1D65
:1089430012AB1178BC12ABCE12AA1D12AA1D12A82B
:108953000F12AB1178B412ABCE12AA1D785812AB1A
:10896300DA785412ABCE12AC74783C12ABDA78548A
:1089730012ABCE12ACAC785412ABDA783C12ABCE5D
:1089830012AB1112AA1D12AB1178BC12ABCE12AAF4
:108993001D783C12ABDA7F3E7EC07D007C0012ABBB
:1089A30011783C12ABCE12AA1D12AB117F3F7E0091
:1089B3007D007C0012A80F12AB11783C12ABCE12D3
:1089C300AA1D12AB117F3F7E807D007C0012A80F91
:1089D30012AB1178B412ABCE12AA1D787012ABDAB7
:1089E300785012ABCE12AB1112AA1D12AB1178C084
:1089F30012ABCE12AA1D784412ABDA785412ABCE66
:108A030012AB1112AA1D787412ABDA784012ABCEF6
:108A130012AB1112AA1D783C12ABDA7F407E807D27
:108A2300007C0012AB11784412ABCE12AA1D12AB1C
:108A3300117F417E107D007C0012A80F12AB1178CC
:108A43004412ABCE12AA1D12AB11787412ABCE1224
:108A5300AB117F407EA07D007C0012A80B12A80FF3
:108A630012AB11783C12ABCE12AA1D12AB117F3D93
:108A73007E2A7DAA7CAB12AA1D12AB117F3F7E001A
:108A83007D007C0012A80F12AB11785412ABCE12EA
:108A9300AB11787012ABCE12AA1D12AB11783C1237
:108AA300ABCE12AA1D12AA1D12AB11785812ABCE6F
:108AB30012A80F12AB117F3F7E7F7DE57CC912AAFE
:018AC3001D95
:108AC40012AB117F4B7E187D967C8012A80F12ABDF
:108AD4008312AB117FE87E037D007C0012AEA112ED
:108AE400AB3078C8A61208A61308A60608A607780D
:108AF4007412ABCE12AB117F3F7E807D007C0012DE
:108B0400A80B12AB11784412ABCE12A80F12AB1102
:108B14007F3E7E2A7DAA7CAB12AA1D12AB1178403F
:108B240012ABCE12AA1D12AB11783C12ABCE12AA14
:108B34001D12AB11784012ABCE12A80F12AB117FED
:108B44003F7E7F7DE57CC912AB11787012ABCE12EB
:108B5400AA1D12AA1D12AB117F487EF47D247C004D
:108B640012A80F12AB8312AB117FE87E037D007C49
:108B74000012AEA112AB3078C4A61208A61308A640
:108B84000608A607223F3F4344454647484A4B4C04
:108B94004D4E5051525354555657583F3FE4F539B2
:108BA400F5A7908BB5791078B4E493F6A308D9F9B6
:108BB4002232A5C24A4A19DC3A885CDB3BFFD6DC88
:018BC4003B75
:10A79F00D2D58002C2D575A70490040078107F0B24
:10A7AF0012A7CB78267F0512A7CB783C7F2212A762
:10A7BF00CB786A7F0F12A7CB75A7002230D506E69C
:10A7CF00F008DFFB22E0F608DFFB22D2D58002C2C1
:10A7DF00D575A7049006FA78737F0612A7CB75A7D5
:10A7EF000022DA0CD902800BD906303701B350059D
:10A7FF0002A97E923702A96AD9F680F9D236800271
:10A80F00C23612A9AF303606C86002B237C89236C8
:10A81F00DAD0D9E4B8000A12A9F6A236923702A903
:10A82F005360FBB51300400F12A9F6A23692F7A2A0
:10A83F00379236A2F79237C398F40424E740DF2407
:10A84F0019AD29AC28AB277A00C394084008CDCCAA
:10A85F00CBCAE4CD80F424086010F9C3ED13FDECEE
:10A86F0013FCEB13FBEA13FAD9F1A236303701B31D
:10A87F0040308A17E5102BF518E5113CF519E51254
:10A88F003DF51A501A13F51AE51913F519E51813B2
:10A89F00F518E51713F5170513E5137002051402E4
:03A8AF00A909E410
:10A8B200C39AF517E5109BF518E5119CF519E512F9
:10A8C2009DF51A500DB237C378177F04E496F60847
:10A8D200DFFA7A047019E513C39408F513500215D0
:10A8E20014E4C517C518C519F51ADAE802A9AA2091
:10A8F200E7BAE5137002151415137817C37F04E63F
:10A9020033F608DFFA80E8E51A20E7137817C37FE9
:10A9120004E633F608DFFAE513700215141513E5A1
:10A92200173378187F03E63400F6500E08DFF77508
:10A932001A800513E51370020514E51420E754701C
:10A9420027E513604E046020851A128519118518B7
:10A95200105326F0AC10AD11A237E51313FFE51228
:10A9620092E7FEA81302AB30E4F512F511F510F5EB
:10A97200147513FF5326F043260580D8E5FFF51220
:10A98200F511F510751400F513D2375326F043264E
:10A992000980C15326F0432603E4F512F511F510A0
:10A9A200F514F513C23780AC5326F080EC79017AA6
:10A9B200018512F0E513A2F7339237751400F513EF
:10A9C2006002D2F785F012A813B8FF0809E512C297
:01A9D200E79D
:10A9D3006001098C278D288EF0A2F7EF3304700AEB
:10A9E3000AC2F705F00AD5F0011A146002D2F785FE
:10A9F300F02922C88813C512C529C512C511C52857
:10AA0300C511C510C527C51022DA03B8000302A972
:10AA13007ED9028002D9F702A96A12A9AF303701A1
:10AA2300B392377004D9E78005DADEB8000302A9D0
:10AA3300AAD9E2C3947E500215142513F5135002CC
:10AA430005147815760008B81BFA78277915E608F7
:10AA5300FAE8FC78108AF0E608A427F709E5F0374E
:10AA6300F7500989F00907E760FBA9F0B813E61965
:10AA730019ECF8B82AD802A90902A995B8FFFA0275
:10AA8300A97ED9FB02A96ADAF6B800F002A9AA12D4
:10AA9300ABE612A9AF303701B392377007D9E3B8E9
:10AAA30000E280DBDAE1B8000280E1D9D5C8C398BF
:10AAB30050021514247F50020514F513781A7600FA
:10AAC3007A1A7B80C3E5109527E5119528E5129541
:10AAD300294016C3E5109527F510E5119528F511C2
:09AAE300E5129529F512E64BF687
:10AAEC00DA0302A909EB03FB30E703187600C3E590
:10AAFC001033F510E51133F511E51233F51240CA98
:10AB0C0030E7DD80B6E53905396010D0F0D0E0C013
:10AB1C0010C011C012C013C0E0C0F08F138E128D84
:10AB2C00118C1022E539146010D0F0D0E0D013D085
:10AB3C0012D011D010C0E0C0F01539227920800C51
:10AB4C007910800479087D007E007F003392D55007
:10AB5C000312ABC0EC33400FEF33FFEE33FEED339B
:10AB6C00FDEC33FCD9EE22EECCF5F0747E29A2D5A7
:10AB7C0013FF92F7AEF022EF8EF0A2F7D2F73392DA
:10AB8C00D5C3947F5006E4FFFEFDFC2294204004C4
:10AB9C0074FF80F304CCFEE4FFFAE5F0CC6012C342
:10ABAC00CC13CCCD13CDCE13CECF13CF0450EEDAC5
:10ABBC00EC30D5D7C3E49FFFE49EFEE49DFDE49CFE
:03ABCC00FC22E682
:10ABCF00FC08E6FD08E6FE08E6FF22ECF608EDF6C7
:10ABDF0008EEF608EFF622CFC513CFCEC512CECDB5
:10ABEF00C511CDCCC510CC22E4F513F512F511F536
:10ABFF001022E493FCA3E493FDA3E493FEA3E49358
:10AC0F00FFA322C0E012AB1112AA1D12AC4512AC69
:10AC1F0001D0E0C0E012AB1112AC3C12AA1D12AB76
:10AC2F001112AC0112A80FD0E0D5E0E722AC48AD6D
:10AC3F0049AE4AAF4B228C488D498E4A8F4B2274B6
:10AC4F00FF7809FFFEFDFCE52654F048F526221299
:10AC5F00AD0504A2E1927F1420E01590AD86740437
:10AC6F0012AC12802912AD0530E102B27F20E0EB69
:10AC7F008C4C8D4D8E4E8F4F90AD9A740412AC123A
:10AC8F0012AB11AC4CAD4DAE4EAF4F12AA1D307F73
:10AC9F0004EF6480FFEE33EF337001FF2212AD0536
:10ACAF00C0E08C4C8D4D8E4E8F4F90ADBE74031205
:10ACBF00AC1212AB11AC4CAD4DAE4EAF4F12AA1D34
:01ACCF00EC98
:10ACD000C54CFCEDC54DFDEEC54EFEEFC54FFF90DA
:10ACE000ADAE740312AC12D08212AB11AC4CAD4DB0
:10ACF000AE4EAF4FE58230E00712AA95B27F809D3D
:10AD000012AA928098EE33EF3324605007D0E0D03F
:10AD1000E002AC4EEFA2E7547F927FFF12AB117CB2
:10AD2000837DF97E227F3E12AA1DEE33EF3324810C
:10AD3000501012AB1112AB8312AB48EFB2E7FF1207
:10AD4000A80FEE33EF33602A2403F8C313FFEE920B
:10AD5000E7FEE82481E4501A12AB1112AB83EF0432
:10AD6000C2E0FCF58212AB50EFB2E7FF12A80FE58C
:10AD70008203FAEE33EF33600B148FF0A2F713FF68
:10AD8000EE92E7FEEA2283FA703AE4E9AABCF8E020
:10AD9000813EE6E99DBF0000803F1A3C2839666984
:10ADA00099BBE335A33DE75D25BFDB0FC93FCCDB96
:10ADB0008D41EE3649C43F91C9453DF8B0C500000C
:10ADC000803F34F517C373FA2F45DDFD0AC6EF2522
:10ADD00013FFEE3512FEED3511FDEC3510FC02AB24
:10ADE00030C3EF9513FFEE9512FEED9511FDEC9536
:10ADF00010FC02AB30EFF88513F0A4FFE513C5F0AB
:0AAE0000CEF9A42EFEE435F0CDFAE1
:10AE0A0088F0E512A42EFEED35F0FDE433CC85136F
:10AE1A00F0A42CFCE5128AF0A42CFCE51189F0A41C
:10AE2A002CFCE51088F0A42CFC89F0E512A42DFD79
:10AE3A00EC35F0FCE51188F0A42DFDEC35F0FC8A28
:10AE4A00F0E513A42DFDEC35F0FC02AB30E4CCF8B0
:10AE5A00E4CDF9E4CEFAE4CFFB75F020C3E5133371
:10AE6A00F513E51233F512E51133F511E51033F553
:10AE7A0010EF33FFEE33FEED33FDEC33FCEF9BEEC8
:10AE8A009AED99EC98400CFCEF9BFFEE9AFEED9937
:10AE9A00FD0513D5F0C622C2D5EC30E705B2D512AE
:10AEAA00ABC0E51030E70DB2D512AEC412AE5712E0
:10AEBA00ABC0800312AE5730D515C3E49513F51312
:10AECA00E49512F512E49511F511E49510F51022A6
:109FD900E57124885002D2191267DC8E4712964126
:109FE900126B69126B07128E96126A5A123E54123C
:109FF9004941103626301219E412A10B12A1201280
:10A00900A21F12A24130510302A2CB12A59C2051DA
:10A0190009C251E4F552F545F5442274FF12A10B2A
:10A029001267DC8E1C8F1B7510DF751100E511643A
:10A03900B4700612A0D675111012A0A34028AE1C48
:10A04900AF1B12686220321EAC03AB027A0C126499
:10A059008BED701275A700758304851182ECF005EC
:10A0690083E510F00511D510C412A0D675C7037584
:10A07900C6E075A7049005007F0412A091DFFB7567
:10A08900A700123004026B07E0F5BCE0F5BDE0F56E
:10A09900BEE0F5BF124F9805C622E51075F004A47D
:10A0A900F5C685F0C775B901E5BC33401F05C6057E
:10A0B900C675B90185BE6485BF6505C675B90185D3
:10A0C900BC6685BD6785BE6885BF69C322E5112465
:10A0D900FE502E75A7007F10AE111E7583048E8267
:10A0E900E0FD1582E0CDB505005012F00582CDF0F6
:10A0F9000583E0FD1582E0CDF00582CDF0DEDCDFE1
:10A10900D72275A75490040005A79005007FB4F0E5
:03A11900F0DFFC78
:10A11C0075A7002212B66AC2517B077AFFE4FFF5DD
:10A12C00A790040012A203ED244C403275A7008DB9
:10A13C008205A712A1C97583058D82E02410401CED
:10A14C00F005A7E02CF0500505A7E004F0BA000CD0
:10A15C00BB0009D251EF24DC50027F23DFC6EA603A
:10A16C000512A17C8006EB600312A1B475A7002236
:10A17C0030E0047553082230E1047553182230E2A4
:10A18C00047553282230E3047553382230E40475E7
:10A19C0053482230E5047553582230E60475536851
:10A1AC002230E7037553782230E00475538822304F
:10A1BC00E1047553982230E2037553AA22ED54F052
:10A1CC00C4232390A1D3735302FE225302FD2253C6
:10A1DC0002FB225302F7225302EF225302DF2253D7
:10A1EC0002BF2253027F225303FE225303FD22534C
:10A1FC0003FB225303FB2212B57312B476E4F5F77A
:10A20C00C2B2C2B2ADF7F5F7C2B2C2B2ACF7D2B2BB
:10A21C00C2202290050078B4E06015FD54F0C4CD46
:10A22C007C00540FFE1583E0FF126589EFF0058367
:08A23C000582D8E422758304B9
:10A2440078FF088882E060FAF5D38812E512244C7E
:10A2540050012285D3D288D4881279FF0512E512E1
:10A2640060F00908E875F0B484A8F08882E060EC36
:10A27400F5D3B9000280D5B9230050D0C395D2924A
:10A28400D15002F40409FEE4FFFCAD01126596749A
:10A2940001FA25D475F0B484A8F0AC06AB071264B7
:10A2A4007DEB30E7010CE5D22C30D1029C9C8882F6
:10A2B400F00AEAB501DCE512244C50012285D3D220
:10A2C4008512D4A812809390040012A38A8C068B62
:10A2D4000512A38AE4FFF512F5118C148B13C3ED58
:10A2E4009BF9EE9CFA4012E51199E5129A500A8CFA
:10A2F400148B138A1289118F528F82E0F9C3ED995E
:10A30400FDEE9400FEE582245A5002244C75F0B40C
:10A314008485F082E0FA2DFDEE3400FEEB9AFBEC2E
:10A324009400FCE92BFBEC3400FC0FBFB4B0E55205
:0CA3340024D3400224B4F552C3E51333D7
:10A34000FBE51433FCE511FE2BFBE512FF3CFC1290
:10A3500065EBE9F890A39C93F511FDEBF513FFEC89
:10A36000F514FE7C001265898F44E890A49C93FA52
:10A37000AB13AC141264B4AF03AE04AD117C001285
:10A380006589EF7002F552F545227C007B007F5A0B
:10A39000E02BFBEC3400FC0582DFF522B4B4B4B44E
:10A3A000B4B4B4B4B4B4B4B4B4B4B4B4B4B4B3B36F
:10A3B000B3B3B3B3B3B3B3B3B3B3B3B2B2B2B2B272
:10A3C000B2B2B2B2B1B1B1B1B1B1B1B0B0B0B0B07E
:10A3D000B0B0AFAFAFAFAFAEAEAEAEAEAEADADAD97
:10A3E000ADADACACACACACABABABABAAAAAAAAA9BA
:10A3F000A9A9A9A9A8A8A8A8A7A7A7A7A6A6A6A5E6
:10A40000A5A5A5A4A4A4A4A3A3A3A2A2A2A2A1A11A
:10A41000A1A0A0A0A09F9F9F9E9E9E9D9D9D9D9C54
:10A420009C9C9B9B9B9A9A9A999999999898989792
:10A4300097979696969595959494949393939292D4
:10A4400092919191919090908F8F8F8E8E8E8D8D15
:10A450008D8C8C8C8B8B8B8A8A8A89898988888859
:10A46000878787868686858585848484838383829F
:10A4700082828181818080807F7F7F7E7E7E7E7DE3
:10A480007D7D7C7C7C7B7B7B7A7A7A797979787824
:10A49000787777777676767575757474000203052C
:10A4A0000608090B0C0E101113141617191A1C1D8F
:10A4B0001F2122242527282A2B2D2E3031333436F4
:10A4C00037393A3C3D3F404243454648494B4C4E64
:10A4D0004F505253555658595A5C5D5F60616364E2
:10A4E0006667686A6B6C6E6F707273747677787A71
:10A4F0007B7C7E7F80818384858688898A8B8D8E14
:10A500008F9091929495969798999B9C9D9E9FA0D1
:10A51000A1A2A4A5A6A7A8A9AAABACADAEAFB0B1A5
:10A52000B2B3B4B5B6B7B8B9BABBBCBDBEBFC0C094
:10A53000C1C2C3C4C5C6C7C7C8C9CACBCCCCCDCE9F
:10A54000CFD0D0D1D2D3D4D4D5D6D7D7D8D9DADAC0
:10A55000DBDCDCDDDEDEDFE0E0E1E2E2E3E4E4E5FB
:10A56000E5E6E7E7E8E8E9EAEAEBEBECECEDEEEE4E
:10A57000EFEFF0F0F1F1F2F2F3F3F4F4F4F5F5F6B5
:10A58000F6F7F7F8F8F8F9F9FAFAFAFBFBFBFCFC36
:10A59000FDFDFDFEFEFEFEFFFFFFFFFFC251E4F5E5
:10A5A00044F814FB900400A9007C0FC2D112A6B796
:10A5B000E82405F8B8B4F08B13E5122403FA244C10
:10A5C0005001FABBFF012275112C8A1912A6EE8FD9
:10A5D00016203D12AA1975112312A6EE8F157516B5
:10A5E00000303DE2801175112312A69675150030DA
:10A5F0003D05E82F13F51575111212A69675140076
:10A60000303D05E82F13F514EA2404F552244C508C
:10A6100002F552E4F51AF51BF51CE516600AFB7A03
:10A6200000AF137EFF12A65CE515600AFB7A4FAF00
:10A63000137EFF12A65CE516600DFB7A00E5146040
:10A6400006FF7ECF12A65CAE1CAF1B7C00AD1A12BB
:07A6500065898F45EF25131A
:10A65700F544D25122EFF5F0A4FCADF0EBF5F0A4F0
:10A667009CFCE5F09DFDEB8AF0A4FAABF0EF8EF0D1
:10A67700A49AF8E5F09BF9E833F8E933F97B00127F
:10A68700662F051AE51B2BF51BE4351CF51C22EA82
:10A697002511F9244C5001F9C2D112A6B5303D421B
:10A6A7008F00C3EA9511F9500324B4F9D2D17C097C
:10A6B700E4FDFEFF8982E060062FFFE43EFE0D0900
:10A6C700B9B4027900DCEDED20D118F51E24FE9215
:10A6D7003D500F126596EFB503005006851E1FFB10
:10A6E700881222F51D80E612A696203D43740212B9
:10A6F700A78D12A696203D38740412A79512A69628
:10A70700203D2D740612A78D12A696203D227408AF
:10A7170012A79512A696203D17740A12A78D12A6A6
:10A7270096203D0C740C12A79512A696203D012287
:10A73700C3E89F605088148F158A1640081ABAFF1D
:10A747000A7AB380060ABAB4027A0012A696303D96
:0DA7570034C3E89FF9602EC3E5149515FB8F
:10A764006930E7D4E930E703F404F9EB30E702F4A5
:10A7740004C3995002AA16E5142515C82F28FFE42E
:10A78400FC33FE7D04126589222AFA244C5001FA16
:0BA7940022C3CA9AFA500324B4FA2230
:10B3E700C2B212D3EBD2B275F83022C2B2F5F7C2AD
:10B3F700B2C2B2D2B222D220D214740612B3F274FD
:10B40700C712B3F21216FF12B41A124F98801F74A4
:10B41700FF8001E4F5BCF5BDF5BEF5BF221216FFAE
:10B4270085BF6C85BE6B756A0012B493C21FD220AC
:10B43700C2B275F705C2B2C2B2C2B2C2B275F705DF
:10B44700C2B2C2B2C2B2C2B2E5F7540170EFD2B211
:10B45700C22022D220C2B2F5F7C2B2C2B2856CF7BF
:10B46700C2B2C2B2856BF7C2B2C2B2856AF722D244
:10B4770020C2B275F703C2B2C2B2856FF7C2B2C2B9
:10B48700B2856EF7C2B2C2B2856DF722E56B70174F
:10B49700E56A7013D22012B435740612B3F274D869
:10B4A70012B45AD2B2D21FC2202212B435D220749B
:10B4B7000612B3F2740212B45A8FF7C2B2C2B2D2F2
:10B4C700B2C22022852E72E55F030354C0F8E55E01
:10B4D700543F28F57C30550122201F0612B49330C3
:10B4E7001F25D220C2B275F705C2B2C2B2C2B2C21C
:10B4F700B275F705C2B2C2B2C2B2C2B2E5F7540121
:10B50700D2B2C220600122C21F12B79612B435D23E
:10B5170020740612B3F2740212B45A787086F708D0
:10B52700B880FAD2B2C2207410256A54F0F56AE4E2
:10B53700356BF56BE4356C540FF56C22D380F0E571
:10B547004B75F010A4256A54F0F56AE5F080E1E543
:10B557006A24F054F0F56AE56B34FFF56BE56C345B
:10B56700FF80D4E56A24FF80ECC380EBE56D24F00F
:10B5770054F0F56DE56E34FFF56EE56F34FF540F4B
:10B58700F56F22D3E4356EF56EE4356F80F075A75D
:10B59700047583048F827870E6F008B880FA75A77F
:10B5A700002275A7049004B47F20E4F0DFFD80EE4D
:10B5B70012B61112B63DC254C255E57F7002D2557C
:10B5C700147002D254E54A30E00122B4061E20541A
:10B5D7000F12B55612B6E112B77512B7AD02B83DE4
:10B5E700128BCB7E0412D3E7754A012220550F1226
:10B5F700B52E12B75412B79612B6BA02B810128BFC
:10B60700CB7E0412D3E7754A0522740312B45A7825
:10B6170070E4F5F7C2B2C2B2A6F708B880F3D2B2A7
:10B62700C22022740312B45AE4F5F7C2B2C2B2E5DB
:10B63700F7D2B2C22022E575F8541F30E40244E085
:10B64700F57585722EA2779226E57C543F30E50288
:06B6570044C0F55EE57C35
:10B65D0054C02323F55FE57F1414F55122856C6FDB
:10B66D00856B6E856A6D22856F6C856E6B856D6AD7
:10B67D0022E4FEFF740775A704F5838E8274FFF034
:10B68D00DFFD75A7002274067E007FB012B683E43D
:10B69D00F55AF55B2275A704758306E55A600A75A0
:10B6AD00F00A84E5F07002740AC4F5822230772026
:10B6BD00E55A24024002055A12B6A2E55AF0E57386
:10B6CD00F0E574F0E575F0E576F0E577F0E578F006
:10B6DD0075A700223077F912B6A27F1074FFF0DF44
:10B6ED00FDE55A24F5500312B70C155AE55AB4FF6F
:10B6FD0002055AC3E55A955B50D6755B0080D11291
:10B70D00B66A7F0A056D056D12B476E4F5F7C2B21F
:10B71D00C2B2E5F7D2B2C22030E704DF02800512D3
:10B72D00B57380E0056D12B47612B6A2E55A24F613
:10B73D00F07F06E4F5F7C2B2C2B2E5F7F0DFF4D25E
:10B74D00B2C22075A70022053FE53FB43C17753FF7
:10B75D0000053EE53EB43C0D753E00053DE53DB4AE
:10B76D001803753D00024BD0153FE53FB4FF17752B
:10B77D003F3B153EE53EB4FF0D753E3B153DE53DAA
:03B78D00B4FF0303
:10B79000753D17024BD00542E542B43C0F7542009F
:10B7A0000541E541B43C057541000540221542E5DF
:10B7B00042B4FF0F75423B1541E541B4FF057541A9
:10B7C0003B154022E54075F03CA42541FBE435F0F3
:10B7D000FC7A3C12647DEB2542FBE43CFC22E53D17
:10B7E00075F03CA4253EFBE435F0FC7A3C12647D08
:10B7F000EB253FFBE43CFC22E54D0475F03C84E581
:10B80000F0653F600312B4CB853F4D2220740122C6
:10B81000C3E5709557FF24FD5021EF24EB400A78D3
:10B82000BD06B6001618068012EF2402400DEF2464
:10B8300014500878BB06B600021806802BC3E570CA
:10B840009557FF24FD5021EF24EB400A78BB16B634
:10B85000FF1618168012EF2402400DEF2414500832
:0CB8600078BD16B6FF021816857057223E
:10D3D40012D3DD12D3DD12D3DD7E0480067E0280FB
:10D3E400027E017F0080047F017E00EF4E6012E424
:10D3F400FD0D1D0DEDC394AD40F7EF1F70ED1E80C4
:02D40400EA221A
:10D4AD00D22FF5D8D2DCE5F520E7FBE5DA540FFEF7
:06D4BD00AFD975D8002272
:10D16F007F767E06909676127318740412D4AD7C77
:10D17F00007D52126589EFF875F00A84C0F07F7652
:10D18F007E2312C9C37E29742E12C9D67E2ED0E0FB
:10D19F0012C9C37E35745612C9D67F6B7E1190D1DA
:10D1AF00D812CA04E824E04001220423F824E750EF
:10D1BF0002781812D1C8D8FB227F6CE82411FE79AF
:10D1CF000512D4060E0FD9F922071DFFFFFFE080CD
:10D1DF00000020C0000038E0000008F0000038F820
:07D1EF00000020FFFFFFE03C
:10D1F60012D21E30E6022409540F75F00AA4F51562
:10D2060012D21E30E6022409540F25152212D21E10
:10D21600540F2275F000800875F044800375F007FE
:10D22600E4206D07D5E0FAD5F0F722C2ACE54F62EF
:10D236003885504F8599509247A26E926DA26F9293
:10D246006EC26FA247D2AC2212D258C4FA12D2587A
:10D256002A2212D21E20E603540F22540724092242
:10D04B00E612D05218E608FAC412D058EA540F442C
:10D05B0030F924C6E950112407800D75F00A84C0FD
:10D06B00F012D071D0E0443030530975F00085E0F8
:10D07B00E0D5F0FA3099FDC299F599623822E5387E
:10D08B0080F2E53812D052800812D073E53812D0F6
:10D09B0073740D12D073740A80CE744012D07374F3
:10D0AB004080C5742C80C1742E80BD12D0CEE91285
:10D0BB00D07F800312D0CEE812D07FE53812D07F1C
:10D0CB000249C11249C180031249D9744075380015
:02D0DB0080963D
:10D4D50085A0835383FE438380858384F075840010
:01D4E5002224
:10CFAF0074A212D4D574A112D4D574C012D4D5746E
:10CFBF002512D4D512D03175C70375C6FC75B901CA
:10CFCF0012D00224EA50027E16EE90D01A9325BC9E
:10CFDF00FE24E6501A24E84016748112D4D5EE12BE
:10CFEF00D4D512D03E742F12D4D574AF02D4D57EBF
:10CFFF002680E6740812D4ADEE75F020A4FEEF542F
:10D00F00F80303032E2492C313FE22F7F7F8F8F95F
:10D01F00FAFBFCFDFEFF000000000101020202030B
:10D02F000303A8BCA9BDAABEABBFACC7ADC62288BF
:0CD03F00BC89BD8ABE8BBF8CC78DC62289
:10D30F00D21AC006C007C0E075A7019000007EB713
:10D31F0075A700EE12D4D5741012D4D5740412D49C
:10D32F00D585A08343838185838475A7517F80E052
:10D33F00F0DFFC1EBEAFD9E4F5A7F584D0E0D0072F
:05D34F00D006C21A2205
:10D4C30075A711900000E4C583F0C58330E2F8F539
:02D4D300A7228E
:10D40600EF20E723EE20E71F20E61C05A7C4540300
:10D41600F583EE5408C42FF582EE5407240983F5EC
:10D42600F0E045F0F005A722804020100804020134
:10D43600EF20E723EE20E71F20E61C05A7C45403D0
:10D44600F583EE5408C42FF582EE5407240983F5BC
:10D45600F0E055F0F005A7227FBFDFEFF7FBFDFEFA
:10C98300FDA42582F582E5F03583F583ED22906FD2
:10C99300737A0475F00512C9837D0580607A05807A
:10C9A300027A04547FC0E0C083C082C39420500144
:10C9B300E4906F2312C996803090707C7A058005CD
:10C9C3009071327A0675F00712C9837D07802E7A3B
:10C9D3000580027A06547FC0E0C083C082C39420DE
:10C9E3005001E49070C212C9C8D082D083D0E02233
:10C9F300906EA175F00A12C9837D0A7A07C2D180AD
:10CA030002D2D1C0A7C082C083C007C006C0E03035
:10CA1300D10975A704E493FDE493FAEEFB75A7042B
:10CA2300EBFEEAFC7901D9067908E493F5D4E5D461
:10CA330023F5D420E01612D4360EDCEA0FDDE1D064
:10CA4300E0D006D007D083D082D0A72212D40680AC
:10CA5300E8906DE175F00E12C9837D0E7A0812CA53
:10CA630000906E8975F00212C983E493FDE4A393E9
:10CA7300FACE2408CE7C0812CA817C06AD02ED23CF
:10CA8300FD20E00712D4360FDCF42212D40680F71F
:10C86E00F5D2C2D58036F5D2D2D58030F5D224F6A7
:10C87E0050090E0E24A650030E0E0EE5D2F5D275FB
:10C88E00F0648485F0D3C2D57009D2D5742012C954
:10C89E00D6800312C9C3CE2406CEE5D375F00A8422
:10C8AE0085F0D3700A30D507742012C9D6800312D2
:10C8BE00C9C3CE2406CEE5D312C9C3E5D222F5D222
:10C8CE0075F0648485F0D3C2D58022F5D2C2D580AE
:10C8DE0025F5D2D2D5801FF5D275F0648485F0D3BC
:10C8EE00C2D57009D2D5742012C9D6800312C9BC24
:10C8FE00CE2405CEE5D375F00A8485F0D3700A30C8
:10C90E00D507742012C9D6800312C9BCCE2405CE19
:10C91E00E5D312C9BCE5D222F5D2C2D58035F5D207
:10C92E00D2D5802F30E70DF404C0E0742D12C9A4C7
:10C93E000E0ED0E0F5D275F0648485F0D3C2D570BA
:10C94E0009D2D5742012C9A4800312C991CE240431
:10C95E00CEE5D375F00A8485F0D3700A30D507740E
:10C96E002012C9A4800312C991CE2404CEE5D3129D
:05C97E00C991E5D22281
:107300007E008014D23C8002C23C7405FEF51EE46F
:10731000FFF51DF51F203C3375A700E49370012293
:10732000A3B40204051D8003B4010A051FEF24095C
:10733000FFAE1E80E612C9D67D06B440027D03B4BE
:1073400021027D02EE2DFE80D27E0075A700E4931F
:10735000700122A3B40204051D8003B4010F051FB0
:10736000EF2407FFAE1E80E612C9A08008B45B00C0
:1073700050F612C9A40EB4210280D30EB44002808C
:10738000CDB42C0280C80E0EB45F0280C1B45B0085
:1073900040BC0E0E80B8E60812C9D6EE2406FED513
:1073A00013F42290967B30740990967F307303908B
:1073B000968402731875F019D5E0FDD5F0FA1249DC
:1073C0008712D0A5744F12D0D8744B12D094C32218
:1073D000754B00127413124987D2AC12D219C5F042
:1073E0006024C5F0B440F412D21EB4400312D21E81
:1073F000B44F1C12D21EB44B1612D21E12D21E1241
:10740000D21EC2ACC32212D219C5F070D5054BC230
:10741000ACD32230530975F008D5E0FDD5F0FA223F
:107420007F0375F019D5E0FDD5F0FA12498712D027
:10743000A5745712D0D8745012D073748112D073BF
:02744000E56302
:1074420012D073E56212D07378D0E612D07308B806
:10745200D7F8E6F8795F30E702792FE912D0731294
:10746200D07312D07312D073745812D07374431243
:10747200D073E412D073E8C2E775F00A84C425F031
:1074820012D0737864E612D07308B869F8E612D0A5
:10749200941273D0400122DF02800775F0008083CE
:1074A200D250C2ACD322127413C250124987D2AC4A
:1074B2002002EF12D219C5F060E6C5F0B440F11215
:1074C200D21EB4400312D21EB457D7F53812D21EC0
:1074D200B450CF12D21E12D21EF56312D21EF56222
:1074E20078D012D21EF924A0500353015FE924E0A0
:1074F2004002795FA60108B8D8E8780612D21ED8F1
:10750200FB12D21EFC53040FC4540F75F00AA42CB4
:10751200FC249C50027C0078D78601E4B92F02D269
:10752200E72CF6786412D21EF608B86AF812D21E58
:10753200E53860030274A412D21E12D21EC2ACC37A
:1075420022909BA4800390990F7F2012734912D33B
:107552000F02D3E5753400C26B12760E12D3E51218
:107562007986E516600312756E02088D127BEA12A7
:10757200229512D30F10002010010280F81279F127
:1075820050131222A012754310000D10010280F850
:0375920012224280
:1075950080D712777222C26BD22775480A122FF84C
:1075A500753400127AC0753703C26A1239E1106A60
:1075B5000512087E80EA12087E127918127A701276
:1075C5007ACC127BEA12229512D30F1000381001E3
:1075D5000280F81279F1501BE9651560181222A096
:1075E50012754312D3DD10001D10010280F812221E
:1075F5004280C3D26B127A9C7516078559171230D3
:1076050071753500809A02088D12798612763012CE
:107615007ACC7F1912764A909BD17E1212734B7EDB
:1076250023E51602C942909CAD80EF7862E412769C
:107635004178D0745F12764118E4F6227F08F60887
:10764500DFFC227F7B7E007810742012C9A4CE2433
:1076550004FED8F5227F197E0812734B7E28909878
:10766500FB30530390990002734BC26B12763012B4
:10767500767A02088DC251127ACC909BC912765A3D
:107685001222681279867F2012761912D30FE51619
:10769500700512D3DA803675A6FF3051031273BE1A
:1076A500124987D2AC200025306DFA1274AB400C1C
:1076B5001279F14011127772D25180BB105003122A
:1076C5007548C25180D1D25112754380CAC2AC22CD
:1076D500D22775480A122FF8753400C26B127AC08A
:1076E500753703C26A1239E1106A0512087E80E80F
:1076F50012087E127918127A70127ACC1277095014
:01770500D7AC
:1077060002088D90990A12765A12227A12D30FC362
:1077160010001310010510020E80F41274204001AF
:107726002212754880DDD3C2AC22D227C26B7548BF
:107736000A122FF8753400127AC0753703C26A121E
:1077460039E1106A0512087E80EAD26B12791812A6
:107756007A7012794075B901E5BCB2E7F5BC124FF3
:107766009875160785591712307180C8D26B127A30
:107776009C127957E51775F01084240AF54824E819
:10778600500375480A12300485585922D2207532A2
:107796000012B67E75A70490070075150012794091
:1077A60075B901E5BC20E705E515F0801004600D0C
:1077B6006482600975BCFF75B90575B9020515E5E2
:1077C60015242050D8E58224FE400302786DA88255
:1077D600187F0075A7007583078882E0FE75F004A0
:1077E600A41278EBA9BCAABDABBEACBF1582E0FD66
:1077F60075F004A41278EBC3E995BC404C7052EACC
:1078060095BD4045704BEB95BE403E7044EC95BF30
:107816004037703DEE75F004A4041278EBA9BCAABB
:10782600BDABBEACBFED75F004A4041278EBC3E9A2
:1078360095BC4015701BEA95BD400E7014EB95BEC5
:047846004007700D7A
:10784A00EC95BF5008EEF00582EDF01582E58260F6
:10785A0009C3EF958250030277E10FC3E89F400303
:10786A000277D975A70490070075C70375C6A8E003
:10787A00F5BCE0F5BDE0F5BEE0F5BF75B90575B933
:10788A000205C6E58224204006E5C6242050E00809
:10789A0075C70375C68075B901E5BC1278D5F5BC04
:1078AA00E5BD1278D5F5BDE5BE1278D5F5BEE5BFC2
:1078BA001278D5F5BF75B90205C6E5C6245850D663
:1078CA00E5320470FB75A700C22022B4FF0122F939
:1078DA0075A704900700E582686005E06970F7E91A
:1078EA0022F5C685F0C775B901E5BC645F700375FA
:1078FA00BC27E5BD645F700375BD27E5BE645F7094
:10790A000375BE27E5BF645F700375BF272275C77D
:10791A0003E54875F004A42480F5C6E55975F0041A
:10792A0084A8F00825C6F5C675B901A9BCAABDABDD
:10793A00BEACBF861522E515242050037515DFE578
:10794A001575F004A454FCF5C685F0C722E5172482
:10795A00204028E51775F00484A8F00824A8F5C685
:0E796A0075C70375B901A9BCAABDABBEACBF01
:10797800A61589BC8ABD8BBE8CBF124F9822E4F530
:1079880016F51579FF12794075B901E5BCB4FF0405
:107998000516A9150515E515242050E9891579FF5F
:1079A80075C70375C6A875B90109E5BC04601B094C
:1079B800E5BD04601509E5BE04600F09E5BF046074
:1079C8000905C6E5C6242050DD0989172275160069
:1079D80075150112794075B901E5BC20E702051655
:1079E8000515E515242050EB227900E975F004A46B
:1079F80054FCF5C685F0C775B901E5BC20E73078B9
:107A0800D066702B08E5BD66702508E5BE66701F58
:107A180008E5BF66701905C675B90108E5BC66704A
:107A28000E08E5BD66700808E5BE667002D3220937
:107A3800E9242050B6C322127A5F127A47A8017F40
:107A480008E0F608DFFB22127A5F127A57A8017F56
:107A580008E6F008DFFB2278D0796275A704758301
:107A680007EBC454F0F5822212794078D0127A8A52
:107A7800E5BCF9C23C20E702D23C127A8A7862124D
:0A7A88007A8A75B901A6BC08A6BDF4
:107A920008A6BE08A6BF0805C622D22012794078E1
:107AA200D0127AAE127AAE7862127AAE86BC0886AC
:107AB200BD0886BE0886BF08124F9805C622126B03
:107AC2000712D4C3128CFC02D30F12D4C37F007EE0
:107AD20009909BB61273187F0A7E12E5150412C82C
:107AE2007A7F1412C1AE1222427F277E08751307D5
:107AF20078D0127396E6793E30E702792F7E34E928
:107B020012C9D67F3D7E01909CC912734B20311B56
:107B1200303003128104C23B127D7C127B32D23B95
:107B2200127D7C127B44127DC3807C12B86C80E68D
:107B3200C23B7F447453201702744E7E0012C9D692
:107B42008017D23B7F4F745720170274457E001274
:107B5200C9D67E06E51E12C9C37E0CE51D12C9C335
:107B62007E12E51C12C9C37E17746412C9D67E1C2C
:107B7200E51B12C9C37E22E51A12C9C37E28742EE0
:107B8200302602742712C9D67E2DE51912C9C37E8A
:107B920033E51812C9C37E39302607742C12C9D2B4
:107BA2007E3BE53702C9C3742D201702742B7F7008
:107BB2007E1512C9D6127BC77E3A12C8237E019067
:107BC2009CEE0273187E1BE51C12C9C37E21E51BC5
:107BD20012C9C37E27E51A12C9C37E2DE51912C93F
:0B7BE200C37E33E51802C9C3127C68A3
:107BED00127C93127F6A127ACC127FC220171E105C
:107BFD00021B124A2112BFDB127C5012224D7F3420
:107C0D007E2F1273A3127B0512D30F80E212224234
:107C1D00203026203128C23B127D7C127CA878664C
:107C2D00127E7CD23B127D7C127CBD7869127E7CEB
:107C3D00127DC3127D37027F1F1281CD80F212B8E3
:107C4D008180EDE57D75F01084AAF075F00AA42A07
:107C5D00547FFA78D7E654802AF6227F277E08795A
:107C6D00D08700C001D224B9D002C224128049D0DD
:107C7D0001A70010230909EE2406FEB9D7E3221946
:107C8D00EE24FAFE80DB7E3479D7E7A2E792171255
:107C9D007FF679D7E7A21792E7F722C224C23B7588
:107CAD001E007F447E00128006801E1023ED802A68
:107CBD00D23BC2247F4F7E0012800ED2247E06E579
:107CCD001E12803BF51E1023E7D2247E0CE51D12FB
:107CDD00803BF51D303BD41023E1D2247E12E51CF0
:107CED0012803BF51C1023E17E1CE51B12803BF539
:107CFD001B1023E67E22E51A12803BF51A1023E8AD
:107D0D007E2DE51912803BF5191023E87E33E51819
:107D1D0012803BF5181023E87E393026027E3BE5B4
:107D2D003712803BF5371023E3227F707E15127FCB
:017D3D00FE47
:107D3E00C2247E1BE51C12803BF51CD2247E21E55D
:107D4E001B12803BF51B1023E77E27E51A12803BA2
:107D5E00F51A1023E67E2DE51912803BF519102336
:107D6E00E87E33E51812803BF5181023E82278D709
:107D7E00E6C2E775F00A847866F537303B05786918
:107D8E0085F037127DEC30262BE53775F003A40411
:107D9E000475F00584FBE51975F00AA4251875F035
:107DAE0006A42BFBE435F0FC12669FF53712669F96
:107DBE00F5188B1922E563FC339217AB6250031250
:107DCE006710305C0A7AD212648B784012662DAE40
:107DDE0004AF037C277D101265968F1C8037E6FD5D
:107DEE0033921718860418860350031267187A09FF
:107DFE00792778C012662A8B1EADD3ACD2AB06792A
:107E0E00EA78601266288B1DAF06AED27C177D70A5
:107E1E001265968F1CAF05AE047C037DE812659645
:107E2E008F1BAF05AE047C007D641265968F1AED34
:107E3E0075F00A84F51985F01822EC339217500369
:107E4E00126710751D30301786751D2D8081784292
:107E5E007B607CEA800678407B207C4E12B94C79A0
:087E6E002778101266288B1C16
:107E7600AF06AED280AB30262AE51975F00AA425E6
:107E86001875F00AA42537FBE435F0FC7A05126470
:107E96007D8C068B077C007D031265898E048F031B
:107EA600127DB6E51E75F00AA4251D75F00AA425F7
:107EB6001C75F006A4251BFBE435F0FC7A0A126457
:107EC6007DEB251AFBE43CFC7A0A12648BEB251940
:107ED600FBE43CFCE43DFD7A0A12649DEB2518FBAD
:107EE600E43CFCE43DFD301703126718A60518A60E
:107EF6000418A60378D7E6A2E7923DC2E775F00A12
:107F060084FCABF0303B0EAB37EC75F00AA42BA229
:107F16003D92E7F622AC3780F0127F3A305C0A7A5F
:107F26004012648B78D212662D3017031267108CBC
:107F3600638B6222127F4A7A0A12647DEB2518FB54
:107F4600E43CFC22E51C75F00AA4251B75F00AA486
:107F5600251AFBE435F0FC7A0A12647DEB2519FB41
:107F6600E43CFC22127F9C12D3E1C202C223127FA0
:107F76009C10000810010510021B80F51031ED1051
:057F8600300D1026047F
:107F8B00D22680E3D230C23180DDD231C23080D7ED
:107F9B00227F35909CB2127349909CD020300F9069
:107FAB009CE6203109909CC1202603909CB91F7E32
:107FBB001712731802D30F7F357E019098DA127364
:107FCB004B7F347E3A1280EB744E12C9D612D30F0C
:107FDB0012D3E1C2027F347E3AD217751159751252
:107FEB004E802675112E751227801E75113E751247
:107FFB002F801675112B75122D800E75114E751263
:10800B005380067511457512571280EBE511301729
:10801B0002E51212C9D612D30F1000081001051079
:10802B00020B80F5D23C1017E3D21780DF0280E6FB
:10803B004430F8128045E8540F22C2218002D2212D
:10804B00A224922292231280EBE830E709D23C74EF
:10805B0030302102745FF812C9D612D30F100034DE
:10806B0010010510025D80F5D23C102266102367CB
:10807B00B43909745F2021DF743080DBB45F047482
:10808B002D80D4B42D04744180CDB45A0474308047
:10809B00C60480C3D23C302406102237102338B4D8
:1080AB004104742D80B1B42D04745F80AAB45F04B5
:1080BB00743980A3B43009745A20219B743980978A
:1080CB00148094B47108D223E812C9D6800DF8C27B
:1080DB0023800874718001E8028062908100800324
:0380EB009080FC86
:1080EE00C007EF2408FF12CA04D00702D30F0205FF
:0680FE00F8F80205000085
:10D2660075A70090D29875F02D84C2D5C2D16017EB
:10D27600D2D1146007D2D514600DC2D1E5F093FC6B
:10D28600742D95F093FB22E5F093FB742D95F093A6
:10D29600FC220009121B242C353E474F586068704B
:10D2A6007880888F969DA4ABB2B8BEC4CACFD4D9B5
:10D2B600DEE2E6EAEDF0F3F6F8FAFCFDFEFFFFFF2C
:10D35400D23D8002C23DED8BF0A430E70205F0C35C
:10D36400E895F020D50425F025F0FEED8CF0A430EE
:10D37400E70205F0C3E995F030D10425F025F0FF6C
:10D38400203D0B2487500122EF24CC40012202D4FB
:01D394000692
:10CF1200203A437E1C7F5312D4067F5912D4061E38
:10CF22007F5712D4067F5512D4067E2312D4067F71
:10CF32005712D4061E7F5912D4067F5312D4061FED
:10CF42007E2012D4067F5A12D4067E1E12D4067F89
:10CF52005212D406800A7E1C7F5390CF9812CA04C4
:10CF620030741CE5716018E57012D266781F79562C
:10CF72007D0912D358303A0312CF820DBD16F32227
:10CF8200C0060E30D5021E1E12D406D0061F30D1A6
:10CF9200020F0F02D406070700386C446C380005F4
:0DCFA200052070D8702005057088A88870E3
:10C0000030122D909CF87F717E2F12734B12B66AFE
:10C010007A0AC23D12C272203D16DAF812C1747C4F
:10C02000007D03126589EFA2D17E237F6512CA9B32
:10C03000227F567E0512C1BA7F3D12C1CD7F6F129D
:10C04000C1CD7E1F7F4112C20A7E0A7F4112C22CDF
:10C050007E227F5912C22C2012012212B66A857AE2
:10C060001D855E1C857B1B855F1A7AC0C23D12C28E
:10C0700072BAB7048C1C8D1D203D5212C1747C0015
:10C080007D1412658974562F20D1029F9FFF24CB07
:10C0900040028037EF248850028030EA1475F003A4
:10C0A00084FE12D406C3E51B957BFEE51A955F92CC
:10C0B000D55004EEF404FEEEC313FE24E0400C74ED
:10C0C0001F2E30D5029E9EFE12D406DAA120120148
:10C0D000227F5212C16A7F5A12C16A751600751703
:10C0E00053801E201201227F157E2D742012C9D686
:10C0F0007E2D7F1C12D4360EBE40F975162F751793
:10C1000015AC1CAD1D12C1747C007D03126589EF56
:10C11000A2D1AE16AF1792D175F080305C04F5F065
:10C120008001A4A2E792D5E5F075F03284F8E5F03D
:08C1300075F00584C0E0E5F0A4
:10C13800A2D533C0E0E8601E12C9BCEE2406FED0CA
:10C14800E0F8D0E012C9BCEE2405FE742C12C9D662
:10C158000E0EE802C9BC742B20D102742D12C9D668
:10C1680080D97E1112D436DEFB02D436C3ED957A1F
:10C17800FFEC955EFE92D150031267002212B66A58
:10C18800857A1D855E1C7A0AC23D12C272203D0660
:10C19800DAF88C1C8D1D227F1512C1A67F327E3ED7
:10C1A80012D406DEFB227E0E12D4060EBE31F92210
:10C1B8007E0112D4060E0EBE3FF8227E3312D4063C
:10C1C8000EBE40F9227E047D1112D4060E0E0EDD3D
:10C1D800F81F1F7E35909CFC305C057E31909D00D9
:10C1E80002734B7405305C097E32740112C9917474
:10C1F800067E3612C9917E3A740012C9917E3D02BC
:10C20800C9917D0F12D4060F0F0FDDF8227F737DC1
:10C218000380047F727D0512D4060FDDFA227F7138
:10C228007D0780F37D0A12D4060E0E0F0FDDF7226C
:10C23800203D071240077003D23D22056D12B476E7
:10C24800E4F5F7C2B2C2B2ABF7F5F7C2B2C2B2E5D3
:06C25800F7FA30E411EBDF
:10C25E00251DF51DE4351CF51C0519EA30E3010E0C
:10C26E00D2B280117803203D071240077003D23DF1
:10C27E0022D8F3056DE56D2409F56D12B476E4F55B
:10C28E00F7C2B2C2B2ADF7F5F7C2B2C2B285F71BB2
:10C29E00F5F7C2B2C2B2E5F7FCD2B2C220543F30BB
:10C2AE00E50244C0CC54C02323F51AE56D24F6F5FF
:02C2BE006D22EF
:10D0DD007E017F0990D15B12CA042051097E037F26
:10D0ED0000743F02C9D6E4FEFFC3E54512C54DFDF0
:10D0FD00940AED403D9464ED4002746312C8747E51
:10D10D00017F09E552240575F02D84AAF075F0050F
:10D11D00A4CA75F00B842A90D1469312D266BCB87E
:10D12D00027BB87D04EE2DF8EF2DF90D12D354DDF1
:10D13D00FB227E0312C9C380C6000C1622222D3994
:10D14D00444F4F5A66707C7C87939EA9A9000909AC
:10D15D000800410000000000888000000000410030
:02D16D000800B8
:10C54D00305D0A75F08AA42480E5F03400227F0066
:10C55D002074147E110F90C5E712CA047F0A7E0A5B
:10C56D00E52E540702C88B7E0BE571B4FF2DE55106
:10C57D0024025003755100E55112C54D75F005A407
:10C58D00ACF0FB1264537E0D781CE66004E612C914
:10C59D00BCEE2405FE18B818F4800612C54D12C85D
:10C5AD007A7F0C7E11E571602B0EE57064B460240A
:10C5BD0064B475F03284C0F012C9BCCE2405CED05F
:10C5CD00E075F00584C0F012C9BCCE2405CED0E0D4
:10C5DD002302C9BC908E88027318070FFFFF9EE7D8
:10C5ED00AD6B9C6BAD6B9D67FFFF75548030745DBB
:10C5FD0078BD79BBE6FC27FB1819E6FD37F9EBF89A
:10C60D007B0012662F8B547F087E11A80690C65BA7
:10C61D0012CA0430100F20730C7F0A7E1712D43605
:10C62D000E0E12D436E5542483E554500224FA75C7
:10C63D00F01984FB90C6639328FEEB90C66D93FDB5
:10C64D0012D4060F0F12D4061F1F0EDDF322030F97
:10C65D000100FFFE03800000000007070D0C0B0A10
:10C66D0005040302010102030405E57E7001227F2A
:10C67D00357E00746F12C9D67E06E57E12C54D0259
:10C68D00C8E5202C012290C69902CA04050EFFF0C0
:0CC69D00E01CF004F81CFFF03012012239
:10C6A9007F6E7E0090969612CA047F1512C1A67FEE
:10C6B9001F12C1A67F2912C1A67F177E06E53F304A
:10C6C900E00B909D10305C03909D2480132074072B
:10C6D9007E019096B68009909D05305D03909D1A64
:10C6E900127318307306E54E6002154E205718E58F
:10C6F9004EB401131216F5C3E55C9560F5BCE55D12
:10C709009561F5BD124F987F217E01E53F30E01E0E
:10C719003057059097A48020E54E70059097B0801A
:10C72900179096C21273187E30E54E02C8DF302B7F
:10C739000AE54E7007909D2E12731822909D39803C
:01C74900E30C
:10C74A001264257F207E05751900781DC2D5E63052
:10C75A00D51712C9BCEE2405FE18B818F17E1F744D
:10C76A0063305C02746502C9D67005B8191880E294
:10C77A00D2D5CE24FACE746B301702742D12C9D6D4
:10C78A00EE2406FE80C8742012C9D280C87F007EBB
:10C79A0023AC5EAB7A126425781DC2D5E630D50C7F
:10C7AA0012C9C3EE2406FE18B818F1227005B8198A
:10C7BA001680EDD2D53017E4CE24FACE742D12C9E4
:10C7CA00D6EE2406FE80D5742012C9D680D512640E
:10C7DA0025781DC2D5E630D51612C991EE2404FE7D
:10C7EA0018B818F10E745E305C02742702C9A07082
:10C7FA0005B8191680E3D2D53017DACE24FCCE74E8
:10C80A002D12C9A4EE2404FE80CB742012C9A48080
:10C81A00CBC23D12C82E0F0F0E0E7463305C027429
:10C82A006502C9D6126425781DC2D5E630D50C1228
:10C83A00C9F3EE2408FE18B818F1227005B81916C3
:10C84A0080EDD2D5301716740BCE24F8CE12C9F368
:10C85A00EE2408FE80D5740C12C9F380D5303DCB86
:04C86A00740A80E5E7
:10CD01007F797E24E55F30E70122AC5F1CAB7B12AB
:10CD11006453E51B700E742012C9D6EE2405FE1271
:10CD2100CD4F800C12CD4FE51B12C9BCEE2405FE80
:10CD3100E51A12C9BCEE2405FE742C12C9D60E0EDA
:10CD4100E51912C9BCEE2405FE745E02C9D6742D24
:10CD5100201702742B12C9D6EE2406FE22E55F309D
:10CD6100E70122AC5F1CAB7B126453E51B700E74B0
:10CD71002012C9A4EE2404FE12CDA8800C12CDA865
:10CD8100E51B12C991EE2404FEE51A12C991EE24A5
:10CD910004FE742C12C9A40E0EE51912C991EE24D9
:10CDA10004FE742A02C9A4742D201702742B12C91F
:06CDB100A4EE2404FE22A2
:10CA93007E257F09A275E579C23D6002D23D92D120
:10CAA30075F080305C04F5F08001A4A2E792D5E52F
:10CAB300F075F03284F8E5F075F00584C0E0E5F038
:10CAC300A2D533C0E0E8602712C9F3EE2408FED0F4
:10CAD300E0F8D0E012C9F3EE2408FE0F0F205A1F2E
:10CAE300746012C9D61F1FEE2404FEE802C9F37452
:10CAF3000C303D06740A20D1010412C9F380CC2006
:10CB03005904742E80DC205804746180D5746280CB
:10CB1300D1A275E579C23D6002D23D92D175F08014
:10CB2300305C04F5F08001A4A2E792D5E5F075F03E
:10CB33003284F8E5F075F00584C0E0E5F0A2D53362
:10CB4300C0E07F3E7E1CE8602012CA54D0E0F8D0DB
:10CB5300E07F3E7E2812CA547F447E32742E12C96F
:10CB6300D67F3E7E37E802CA54303DE0740A20D1B6
:07CB7300010412CA5480D531
:10C2C000E54424F64001227800E5520475F0038429
:10C2D000F9E928FE24C45001FE12C2F812C3041E5C
:10C2E00012D406C3E998FE5003243CFE12C2F81E85
:10C2F00012D40608B81FDA22EE2420FE24C250030E
:10C300002402FE22E824F1E8C2D55006D2D5E8F492
:10C31000241F23FF90C38293CF0493FAE545F5F0E1
:10C32000A4ACF0FB1264B4E544F5F0A49BFBE5F08B
:10C330009CFCEB2420FBEC3400FC24F0500CEB24A0
:10C3400060EC340090C3D293800EEB33FBEC33FCF3
:10C35000EB33EC3390C3A293FAE5458FF0A430E7BA
:10C360000205F0E5F020D502F4042A75F005201945
:10C370000375F00384FF24DF50027F20C374329FD3
:10C38000FF22FF00FF03FA0BF318EA2ADE40CF5822
:10C39000BE73AB8D96A880C068D64FE835F51BFDFF
:10C3A00000FF00080B0E101214151718191B1C1D86
:10C3B0001E1F20212223242526262728292A2A2B2E
:10C3C0002C2D2D2E2F2F303131323333343435365E
:10C3D0003637373839393A3A3B3B3C3C3D3D3E3EB7
:10C3E0003F3F4042444648494B4D4E5052535556AC
:10C3F00058595B5C5D5F60616364656668696A6B20
:10C400006D6E6F7071727374767778797A7B7C7DDC
:10C410007E7F808182838485868788898A8B8B8CC6
:10C420008D8E8F9091929394949596979899999ACE
:10C430009B9C9D9E9E9FA0A1A2A2A3A4A5A6A6A7E9
:10C44000A8A9A9AAABACACADAEAFAFB0B1B1B2B315
:10C45000B4B4B5B6B6B7B8B9B9BABBBBBCBDBDBE4E
:10C46000BFBFC0C1C1C2C3C3C4C5C5C6C7C7C8C892
:10C47000C9CACACBCCCCCDCECECFCFD0D1D1D2D2DF
:10C48000D3D4D4D5D5D6D7D7D8D8D9DADADBDBDC34
:10C49000DDDDDEDEDFDFE0E1E1E2E2E3E3E4E5E58E
:10C4A000E6E6E7E7E8E8E9EAEAEBEBECECEDEDEEEF
:10C4B000EEEFEFF0F1F1F2F2F3F3F4F4F5F5F6F656
:10C4C000F7F7F8F8F9F9FAFAFBFBFCFCFDFDFEFEC4
:10C4D000FFFFE54524FD400122E5520475F0038489
:10C4E000241FFE24C250032402FE12C523EEFD24A5
:10C4F0001EFE24C250032402FE12C523E54424027A
:10C5000075F00520190375F00384F4042432FF2428
:10C51000EE500F12C518AE051E1E7C0512D4060E75
:10C52000DCFA227F1512D4060F0FBF2DF822E55337
:10C530000475F00384241FFE24C250032402FE125B
:0DC54000C5430E7F2312D4060FBF2DF92234
:10CC3F007E397437301902745512C92C801C75A7B0
:10CC4F00007E007F2F90CCDC12CA04205DE27E357F
:10CC5F00746430190274A012C94230745A301257DA
:10CC6F00E54AB4040122B4060122E57112C36BEF49
:10CC7F00FDE5700475F00384241EFE24C2401F24BA
:10CC8F0003501E90CCC7600990CCCE14600390CC9B
:10CC9F00D5E493A3B4FF0122FE12CCBB80F3240290
:10CCAF00FE7C04EDFF12CCBB0EDCF822EDFF12D49C
:10CCBF00060FEF24CE50F7223B3C3D3E0001FF3CD8
:10CCCF003D3E010203FF3E3F01020304FF053870A2
:10CCDF0001100240078080011003400400600150E2
:10CCEF0003C0070017FCA7FADFF43FE000A00240E3
:02CCFF000780AC
:10D2C600AF177E00E53C12C86E7E0C742E12C9D6CE
:10D2D6007E12E53B12C86E7E1E742E12C9D67E24BF
:10D2E600E53A02C86E7E0E78ADE612C8D97E18748D
:10D2F6002C12C9D67E1B18E612C8D97E25742C12AC
:09D30600C9D67E2818E602C8D938
:10D395007F797E16743B12C9D27E18E53F12C8D933
:10D3A5007F797E0078AEE612C8D97E0A743B12C931
:10D3B500D27E0CE53E02C8D97F797E00E54012C8D1
:0FD3C500D97E0A743B12C9D27E0CE54102C8D949
:10CE6A00787512CEBA7453201702744E207406E5F0
:10CE7A002E54074430AF1712CEE47E3BE57DC454EE
:10CE8A000F12C9C32074077E07742012C9D6787896
:10CE9A0012CEBAE5172409FF7457201702744520E9
:10CEAA007402742012CEE47E3BE57D540F02C9C39E
:10CEBA00E6FD3392171886041886033017031267A3
:10CECA0018791778701266288B13AF06AED27C00D9
:10CEDA007D641265968F148D15227E0012C9D67E46
:10CEEA0007E51312C88B7E19746412C9D67E20E531
:10CEFA001412C86E7E2B742E2073030E742C12C962
:08CF0A00D67E2FE51502C86E6A
:10CB7A00C234E54A603B7A2420E00E7A2614146017
:10CB8A00087A28141460027A297F717E00303F0ADD
:10CB9A00E537640260047F6B7E05EA12C9D6205528
:10CBAA0005205406800B745B8002745C7E0012C9F7
:10CBBA00D630262CC22690CBFF7F681273007F6680
:10CBCA00A85AE54AB4060108E875F06484740AC5EF
:10CBDA00F084C0F012C9F3EE2409FED0E012C9F3C2
:10CBEA00200811E537B402032041097F367E2E74EE
:10CBFA004112C9A4224D41524B00302B0D30430A39
:10CC0A007F707E0190CC15127318224C4F4747450E
:10CC1A0052404641494C00E54375F008A495355009
:10CC2A0013E59020E20ED2347F6F123E4A0F90979E
:05CC3A0007127318222F
:10CDB70020144F740512D4ADEF33EE33F9EF0303AC
:10CDC700541FF5F090CE0AE993A4C5F013C5F013EC
:10CDD700C5F013C5F013C5F0135403FCE5F013FBBE
:10CDE700E9242093C9244093C39BC4540FFBE99CB7
:10CDF700C4FC540FF9EC54F02B2446F57BE934F6C8
:10CE0700F55F22FFFFFFFFFFE6C5AD9C8F857D77AE
:10CE1700726E6C6A696A6A6C6F747A828D9DB4D916
:10CE2700FFFFFFFAE9DCD3CEC9C6C3C0BEBBB9B7A3
:10CE3700B5B4B2B0AFADABAAA8A6A4A2A09E9C9968
:10CE470096918C00381CE735D137246F00C5B3C1E4
:10CE5700E61F66B60E68C21867AADBF4EDB9467519
:03CE670010A20016
:10D48D00D2A27408D2A1D2A300C2A3C2A1D2A3007A
:10D49D00C2A3D5E0EF7405D2A300C2A3D5E0F82254
:10D46600C2A3D2A2D2A1D2A300C2A375F00833925E
:10D47600A1D2A300C2A3D5F0F5C2A175F003D2A331
:07D4860000C2A3D5F0F8225B
:10BC550012D466D2A300C2A3C2A175F008E4D2A390
:10BC650000C2A3A2A233D5F0F5FE75F008E4D2A375
:10BC750000C2A3A2A233D5F0F5FFD2A300C2A3222E
:10BC8500E478806608B88BFB70012274D512BC5528
:10BC95007881C3EE13FEEF13F692D118EE2460F609
:10BCA50074D612BC557888EF33CE33CE33CE33CE2F
:10BCB50033A2D192E25407FCEEFB7A0812647DECC4
:10BCC500244FF608EBF674D912BC55EF543F788231
:10BCD500F67886EF33CE33CE33CE33CE335403F6F8
:10BCE50008EEF618161608E6C4FF54F0F618E6C472
:10BCF500CF540F2FF674DA12BC55EF232354FC787A
:10BD050083F67884EEF608EF54C0F67880E466088A
:10BD1500B88AFBF62212BC5D7889C3EF96FF18EE50
:08BD250096FEA2E792165010F1
:10BD2D00126700740FF8F91264CAEF2CFFEE3DFE96
:10BD3D00788BEEF608EFF622E6182016072CF7E6BC
:10BD4D003D19F722C39CF7E69D80F66A405E80564A
:10BD5D00E050F04B0044803DC0384031D02BA02541
:10BD6D00601F2018D0014401580168017801880135
:10BD7D00A001B401D001EC02100238026802A078D3
:10BD8D00BE8020858E8A9D8F4D95BA9A97A0BEA6AE
:10BD9D0031AC53B22AB801BD6F12BC5D788DEEF691
:10BDAD0008EFF67887798C1264CA7883799012BD82
:10BDBD00457885798C1264CA7881799212BD45785F
:10BDCD008DE624E4FE08E63392D13392D554FCFF80
:10BDDD00EEA2D133A2D533FE780F79921264CA78D0
:10BDED00947990C3EC97F61819ED97F6799490BD68
:10BDFD00587F197D0EEF93C3971F19EF93971F0966
:10BE0D001DED600240EF0F90BD72798DEF93F70934
:10BE1D000FEF93F7788E79941264CA90BD8CEF93DF
:10BE2D00C39BFB1FEF939C2420FC7897E62BF61801
:10BE3D00E63CF618E436F6740612D4ADD237EE248D
:07BE4D00F740062402500239
:10BE5400C237EEFCEFFD740712D4ADC3ED9FFFECC7
:10BE64009EFE78B7E6FD337C0050011CEF2DFFEEFB
:10BE74003CFE78D8E6C4540F2FFFE43EFE789CEFD6
:10BE840026F618EE36F62220141220370F789DE697
:10BE9400B4050912BF2A12BF5F12BFA322201445A2
:10BEA4007897799A12BFBE126688C3EE9420FE92E8
:10BEB4004550031267007C007D05126596304503EA
:10BEC40012670012D0311216EBE5BC2FF560E5BD08
:10BED4003EF5611216F5E5BC2560F57AE5BD3561E0
:10BEE400F55E12D03E7897799AC3E697FB1819E667
:10BEF40097FC7A0212647D30370B7A0212647DEC6F
:10BF0400FEEBFF800312BF2A12BF5F20140312BF8F
:10BF1400A378957998E6F776000809E6F77600089D
:10BF240009E6F7760022799CE77700FB19E77700AA
:10BF3400FC789DE6B40506EB33FBEC33FCECA2E79E
:07BF440092D55003126710B3
:10BF4B007A3212648BECFBEDFC30D503126710ECEC
:10BF5B00FEEBFF22EE2408FE7404203711789DE6D9
:10BF6B00B40504740C8007F42406C323540FFD7C22
:10BF7B0000126469789FE6FC08E6FBC374109DFA17
:10BF8B0012648BEFF8EEF9126688E878A02FF6FFB3
:10BF9B0018EE39F62480FE2292754003126700EFEB
:10BFAB0033EE33F579C276307508E57924F150021A
:10BFBB00D27622E627FB1819E637FC1819E637FD6F
:10BFCB002212B6117F087871793A12BFE7024BD073
:10BFDB00855E63857A62787379647F06E6F7080974
:10BFEB00DFFA227864797380F1787379AF80EB781C
:05BFFB00AF797380E541
:10640300E4FEFFFC7D0A791DE7540F2FFFE43EFEF7
:10641300B9190280061912646980ED3017031267F7
:106423000022305C2BEC3392175003126710EC24DC
:10643300D950047C277B007AD212648BEB33CC33A4
:10644300CD33CC33ED33FBEC33FC30170312671041
:10645300EC3392175003126710791912669FF709EC
:10646300B91DF8A70322EFF88DF0A4FFEDC5F0CE18
:10647300A42EFEEC88F0A42EFE22EB8AF0A4FBE50A
:10648300F0CC8AF0A42CFC22EB8AF0A4FBE5F0CC40
:106493008AF0A42CFCE435F0FD22EB8AF0A4FBE5A2
:1064A300F0CC8AF0A42CFCE435F0CD8AF0A42DFDC9
:1064B30022EB8AF0A430E70205F0E5F0CC8AF0A4E1
:1064C3002CFBE435F0FC2286F0E7FDA4FAABF019CF
:0664D300E786F0A42BFB9C
:1064D900E435F0FC18E68DF0A42BFBEC35F0FCE478
:1064E90033FDE687F0A42CFCED35F0FD22EB89F0B5
:1064F900A4CBAEF08AF0A42EFEE5F03400FDEC89C1
:10650900F0A42EFEE5F03DFDE433CC8AF0A42DFD88
:10651900E5F03CCEFC22EB89F0A4CBAFF08AF0A4E5
:106529002FFFE5F03400FEEC89F0A42FFFE5F03EE3
:10653900FEE433CC8AF0A42EFEE5F03CFCED89F0B4
:10654900A42EFEE5F03CFCE433CD8AF0A42CFCE556
:10655900F03D8E058C068F04FF22C2D5EC30E7058D
:10656900B2D5126708EE30E70DB2D5126700126591
:1065790096126708800312659630D50312670022C8
:10658900C3EC13C0E0ED132FFFD0E03EFEBC000BBF
:10659900BE0029EF8DF084FFADF022E4CCF975F04F
:0465A90008EF2FFFC9
:1065AD00EE33FEEC33FCEE9DEC994005FCEE9DFECA
:1065BD000FD5F0E9E4CEFD22EDF9F5F0EE8420D211
:1065CD001CFEADF075F008EF2FFFED33FD40079980
:1065DD005006D5F0F222C399FD0FD5F0EA22EC3327
:1065ED00EE3400FEEF3400FF7D007A00790078096B
:1065FD00C3ED9AFDEE9BFEEF9CFFB392D54009EDE6
:10660D002AFDEE3BFEEF3CFFA2D5E933F9ED33FD5C
:10661D00EE33FEEF33FFD8D92279007A00C380150F
:10662D0079007A00C3EA13FFE913FEE8132BFBEEA2
:10663D003CFCEF3DFDE4F5D2F5D333FE7F19C3EEFF
:10664D0098FEE5D299F5D2E5D39AF5D3B392D5401C
:10665D000DEE28FEE5D239F5D2E5D33AF5D3A2D524
:02666D00EB330D
:10666F00FBEC33FCED33FDDF0122EE33FEE5D233DD
:10667F00F5D2E5D333F5D380C3EDC454F0FEECC4AB
:10668F00FF540F2EFEEF54F0FFEBC4540F2FFF22D9
:10669F00EC75F00A84FCEB54F025F0C475F00A8415
:1066AF00C4CBC454F025F0C475F00A842BFBE5F07D
:1066BF0022AC10AB1112669FA904AD03FA7C197BB3
:1066CF009912647DAE04AF03EA75F006A4F8AC121C
:1066DF00AB1312669F2875F00A8485F014F8EF2B20
:1066EF00FFEE3CFEEF28FFE43EFEE43DFDE439FC07
:1066FF0022C3E49FFFE49EFE22E4C39DFDE49CFCC5
:10670F0022C3E49BFBE49CFC22C3E49BFBE49CFCC4
:10671F00E49DFD2275D4107B807A0079807800EAA1
:0A672F00F5F0A4FCADF0EBF5F0A4CA
:10673900FEAFF0EB8AF0A4C333C5F033C5F092D5B0
:106749002DFDC5F03EFEE430D501043FFFB5150D22
:10675900EEB51409EDB51305ECB51201224006EAB0
:1067690098FAEB99FBD5D40ABB0001220ABA0001B9
:106779000B22C3E913F9E813F8EA28FAEB39FB808D
:10678900A478087B807D807C00EDF5F0A4FAE5F023
:106799008EF0B5F007EA8FF0B5F001224003ED9BCA
:1067A900FDD827BDFF0122EDF5F0A4F9A8F0ED040D
:1067B900F5F0A4C399FAE5F09813CA1329F9E83A50
:1067C900F8C3E99FE89E50010D22C3EB13FBED2BA3
:1067D900FD80B67473F8F9E627FB0809E637FC086B
:1067E90009E637FD30E703126718EB33FBEC33FC9E
:0B67F900ED3323FD242083F8ED241C69
:1068040083FFED241883FAED241483F9EF99F9E852
:106814009AFA1264F6EF9DFFE89EFE22FFFFFFB690
:10682400FED7FD63FB5DF8C4F59BF1E3ED9EE8CF75
:10683400E379DD9ED743D06BC919C153B91CB07934
:10684400A7709E06943F8A237FB674FF6A045ECBCA
:10685400535B47BB3BF1300423FB17DE0BB2C21D75
:10686400C232752C00C3E5679576FBE5689577FC25
:10687400E5699578FD30E705D26112671824F05078
:1068840003126936AA06A90712651FEC2480E43DA9
:10689400FBF9F51AE43EFCFAF519E43F6002D23242
:1068A4001264F68B128C138D148E15C3E5649573E4
:1068B400FBE5659574FCE5669575FD30E705D262E8
:1068C400126718EBF9F51FECFAF51DED6002D232F0
:1068D400303201221264F6EB2512F512EC3513F571
:1068E40013ED3514F514EE3515F51540E102672363
:1068F40012686220323BEB242E40D3EA2401CB34CD
:1069040000FC7A07793D1264F6C010C0118E108D18
:10691400118C128B13E4FCFD7E077FD012AE5785D9
:106924001203851302D011D010BB0005BA0002D2A5
:106934001D22B261C374809BFB74F59CFC74209D82
:01694400FD55
:1069450022303F647F747E0112C1BA7E1F12C226B7
:1069550075A7009004EDE0A2E792171392E7FC15E6
:1069650082E013FB301703126710BC003BEB603865
:1069750020E73520E63210E513201707C3741F9B67
:10698500FE80027E1F12C21B0EDBFA22FB201709B6
:106995007E00C374209BFB8008EB241FFE74209BA4
:1069A500FB12C2150EDBFA222212BFF475A7007581
:1069B5008307E559C4440FF582E0A2E79252C2E786
:1069C50075F00A84FEAFF075A7045382F17864125E
:1069D5006A31AE077867126A3175A700E57DC45440
:1069E5000FFEE57D540FFF7873126A25AE077876A2
:1069F500126A2574AF1267DE1268F41216E6A9BD95
:106A0500E5597002A9BCE975F00AA4F9EA99900460
:106A1500ECF0A3EB95F0F0A2E7923DD23F02BFFA6E
:106A2500860308860408860518188006E0FBE0FC46
:106A3500E0FD7A0A12649D20E70CEB2EF608E43C93
:0B6A4500F608E43DF622C3EB9EF608C5
:106A5000EC9400F608ED9400F622C23F302A0F783D
:106A6000A87600223038FCC23878C5864622E54830
:106A700024F640EFE5580460EA75A700758307E542
:106A800059C42408F582E070DB0582E0FFE54A6422
:106A9000046015E54A6406600F801DEF24BE50298E
:106AA000C23878C58646802175390AEF20E7097516
:106AB000390520E6037539022038E0EF24C3400988
:106AC000D23878C5A6467546001216E6A9BDE55926
:106AD0007002A9BCE9240DC39F401F1269AE303D6E
:106AE00019753901204006D24078A8762320521625
:106AF000E55965586010D233800C3033090559C20E
:106B000033C2401295FE22E558B4FF012285581188
:106B100075A704758307E54824F65002805C2012AF
:106B200059202905202A02805112BFF4E4F516F5F8
:106B300017751000126B93E510700312BFEE126B05
:106B4000AC302910E51B2517F517F51BE51C35168C
:106B5000F516F51C126BB912BFEE0510C3E51195C1
:106B60001050D175A70002BFFAE55AF51124F6506E
:106B70000375110A75A704758306751000126B93CF
:0F6B8000126BAC126BB90510C3E511951050EEF6
:106B8F0075A70022E510C4F582E0E0F564E0F56535
:106B9F00E0F566E0F567E0F568E0F5692275A701B5
:106BAF00126DA512423575A70422E9F0E51CF0E538
:106BBF001BF022E510C4F582E0F512E5822406F5FC
:106BCF0082E0F511E0F51CE0F51B22305E3A20283B
:106BDF0037E558B4FF012275A704758307E559F50A
:106BEF0010303306655860020510126BC2E0F513C2
:106BFF00E07F7A7E3D12C9A4E5137E3912C9A4E560
:106C0F00127E3512C9A4802C2012012275A704759B
:106C1F008306855B10126BC2E512700B7E3A7F798B
:106C2F00745D12C9D6800D75F06484E5F07E397FEE
:106C3F007A12C926E5376402700830413112948107
:106C4F00802CE51C7006E51B24FB5022E51164B473
:106C5F00601CE51112D266781D79547D1D90CFA16D
:106C6F00E53F20E00390CFA812D35812CA0475163F
:106C7F0019751779E51C24ED402BAE1CAF1B126D57
:106C8F006F7C007D32126596C005EFAF17AE1612FE
:106C9F00C8DFCE2405CE742C12C9D60E0ED0E02339
:106CAF0012C8D9801B126D66126CE1CE2405CE740A
:016CBF002CA8
:106CC00012C9D6CE2402CEE875F0058412C9BCCE16
:106CD0002404CE7422305D02746612C9D675A700F2
:106CE00022EE243D50047EC37F4B7C017DF412656F
:106CF00096C004C005EF6007AF17AE1612C8DFD00C
:106D000007D0067C007D32126596A805EFAF17AE5E
:106D100016CE240ACE02C9BC126D66EE2450305D38
:106D200003EE24A150047EC37F4B7C017DF41265E9
:106D300096C004C005EF6007AF177E2F12C92CD094
:106D400007D0067C007D32126596C005EFAF177E36
:106D50003712C9917E3B742C12C9A47E3DD0E075D8
:106D6000F0058402C991E51B2402FFE4351CFE30C6
:106D70005D1ABEC305BF4D028012AC06AB077A1B7D
:106D800012648B783212662DAE04AF0322787379C9
:106D9000641267E01268F4751CC3751B4B20320443
:106DA0008B1C8A1B22126D8D30320122AC19AE1A57
:106DB000A91DAF1FB90005BC00028010C3E913F97B
:106DC000EF13FFC3EC13FCEE13FE80E8BF29005065
:106DD00006BE2900500122C3EF13FFC3EE13FE804D
:106DE000EB3E7FE3E3E3E3E3E3E3E3E3E37F3E0C54
:106DF0001C3C7C7C1C1C1C1C1C1C1C7F7F3E7FE3E1
:106E0000E3E3070E1C3870E0E3FFFF3E7FE3E3039C
:106E10000F0E0F03E3E3E37F3E070F1F3F77E7E724
:106E2000FFFF0707070707FFFFE0E0E0FEFF0303A0
:106E300003E3E37F3E1E3F73E0E0E0FEFFE3E3E3B6
:106E4000E37F3EFFFFE3E30303070E1C38383838C7
:106E5000383E7FE3E3E37F3E7FE3E3E3E37F3E3ED1
:106E60007FE3E3E3E37F3F030303E77E3C000000AF
:106E7000181818FFFF181818000000000000000084
:106E800000FFFF0000000000003FF00000381C3849
:106E9000F00180C1F020F0FC0038F03FE00000007D
:106EA000007CC6C6C6C6C6C6C6C67C1838781818C2
:106EB000181818187E7CC6C60C183060C0C6FE7C38
:106EC000C6C6061C0606C6C67C0C1C3C6CCCFE0C5A
:106ED0000C0C0CFEC0C0C0FC0606C6C67C3C66C0DE
:106EE000C0C0FCC6C6C67CFEC6C6060C1830303014
:106EF000307CC6C6C67CC6C6C6C67C7CC6C6C67E38
:106F0000060606CC78000018187E7E1818000000CF
:106F10000000007E7E000000000000000000000075
:106F2000000000000000000000000000008080A0C1
:106F3000C0A000304020C08080C0A0A0000060A0A1
:106F4000600000A040A05098D090882050A85088A1
:106F50008850A8502060806000000040E0400000A1
:106F6000000000800000E000000000000040002061
:106F700040800040A0A0A04040C04040E0C0202091
:106F8000C0E0E0204020E02060A0E020E0C0202021
:106F9000C06080E0A0E0E020404040E0A0E0A0E051
:106FA000E0A0E020C0004000400000800080002001
:106FB00060E0602000E000E00080C0E0C080E0E031
:106FC000E0E0E0000000000040A0E0A0A0C0A0C001
:106FD000A0C040A080A040C0A0A0A0C0E080C08011
:106FE000E0E080C080806080A0A060A0A0E0A0A0C1
:106FF000E0404040E0202020A040A0A0C0A0A08011
:10700000808080E0A0E0A0A0A0A0E0E0E0A040A000
:10701000A0A040C0A0C0808040A0A0C060C0A0C010
:10702000A0A060804020C0E040404040A0A0A0A0C0
:0D70300060A0A0A0A040A0A0A0E0A0A0A093
:10703D0040A0A0A0A0404040E0204080E02020A83B
:10704D0070202070A8202008F030D0100000F0A88B
:10705D00A8000000E000000090204870889898403B
:10706D0000E0E0E000A0E0E0E04060301030606063
:10707D009090909090602060202020207060901063
:10708D00204080F06090102010906010305090F0F3
:10709D001010F080E010109060609080E090906093
:1070AD00F010202040404060909060909060609083
:1070BD0090701090600000000000000000000000C3
:1070CD000000005060500070705000007880700813
:1070DD00F000F8888888F800C0C810204098180083
:1070ED00C0B098B0C000602040000000000090D8F3
:1070FD00FCD8900000246CFC6C24000020A870A823
:10710D002000002020F8202000000000000000805A
:10711D00000000F0000000000000000060600008AA
:10712D001020408000708898A8C8887020602020AA
:10713D00202070708808102040F8F8102010088862
:10714D007010305090F81010F880F00808887030EA
:10715D004080F0888870F808102040404070888882
:10716D007088887070888878081060006060006092
:10717D00600000008000008000002040F8402000EA
:10718D000000F800F80000002010F81020007088B2
:10719D000810200020000000000000007088888882
:1071AD00F88888F08888F08888F0708880808088DA
:1071BD0070E09088888890E0F88080F08080F8F802
:1071CD008080F0808080708880B8888878888888F2
:1071DD00F88888887020202020207038101010101A
:1071ED0090608890A0C0A09088808080808080F87A
:1071FD0088D8A8A88888888888C8A898888870881A
:10720D008888888870F08888F08080807088888869
:10721D00A89068F08888F0A09088708880700888A1
:10722D0070F8202020202020888888888888708801
:10723D00888888885020888888A8A8A85088885071
:10724D002050888888888850202020F808102040F9
:10725D0080F800CCAC9CACCC0000CCD4E4D4CC00F9
:10726D0004781828C800FC40A04018202018000001
:10727D0000000000F800000000A040A00000006029
:10728D00006060006000600060600000F0A8A8A8C9
:10729D00A8205020000000005090B890D090886039
:1072AD00505000707050C0A0C090941814304C5CB9
:1072BD006060603C00E0F0080808F88088482818F5
:1072CD00F804008820208870000080C0A090F8008D
:1072DD003048B4B44830003048B4B44830FC00985D
:1072ED00D02058C8008080F088888888F8E8D88039
:0372FD00D8E8F8D6
:0300000002005E9D
:03000B0002AEDA68
:0C000E00206E06859950D26E32D26F32FF
:0E00230010990AC298206DE385994FD26D3274
:10003800E4F537F534F520F52FC229C22AC268C283
:0800480027C214C2150231F1B8
:03005B00022FCCA5
:10AEDA00C0D0C0E0C0F0C0A775A700C083C082750B
:10AEEA00D008758A3D758CEA0532E5327002153252
:10AEFA000530E530640A6026201520E531B40C0BD4
:10AF0A00E530B4010612B26D12CDB7E531B4180BB3
:10AF1A00E530B4060612B26D12CDB702B0E1C2AF87
:10AF2A00D2C075C07AD2AFF5300531E531641970F7
:10AF3A0045F531201522C22C7D0A740412D4ADEED7
:10AF4A0024F540142402400E24014008202005DD87
:10AF5A00E9022FC0D225D22CE5A6600215A678A94F
:10AF6A00E660011678B5E660011678B6E660011665
:10AF7A0078D8E660011620150BE531B40206201ACE
:10AF8A000312CFAF302E09E5367005C22E12B1F486
:10AF9A00E5367004C24B8002153678A8E6600116C1
:10AFAA000535E53570021535E590307B0B30E00844
:10AFBA00D278C27BC200801A307C0B30E108D27989
:10AFCA00C27CC201800C307D0930E206D27AC27D91
:10AFDA00C202E59044F8F4700B753500302D05C2B5
:10AFEA002D12B1F4E5336005153302B086E590F40D
:10AFFA005407700302B086F52075330820001B2021
:10B00A00100C2011098013E59030E10E8006E53717
:06B01A0024FD40F3E543B4
:10B02000541FF53320100375A6FF78A8E67057204B
:10B030002D54202E51301004E536704A20100C207B
:10B040001109E53524F55003753304D21BD2A5D27E
:10B05000A675B40C75B22278A77655C21C053420AB
:10B06000272420682120291E202A1BA2107211509B
:10B0700015E5206011E5342438400B20002620011E
:10B0800019D27D7534C8201558E531702412D48D3D
:10B0900074E812D466802A02B19AE53724FD40E6AE
:10B0A000D27C80DF3011DFE53724FD40D9D27B80B0
:10B0B000D275F00384E5F070DE12BD1A74E812D484
:10B0C00066E531B4060512BE8B8016B40C0512BEBF
:10B0D000A1800EB4120512BE8B8006B4180312BEF6
:10B0E000A1E59020E20620101020110D78A8E6704E
:10B0F0004920103120113280562027F02068ED20A1
:10B1000029EA202AE7E534243140E1240450DD9087
:10B11000B12193D2A6201002C2A6D2A512B1E78017
:10B120004AC8A08267E5367011E59020E221E54328
:10B1300075F009A495355017D22DD2A6201002C261
:10B14000A6D2A57418304B02746412B1E7801C209B
:10B15000340E305A08E54A603C1414603812B1F4D9
:10B16000101B08A25892A5A25992A675A700D082DA
:10B17000D083D0A7D0F0D0E0D0D0202006C5A660E4
:01B1800003CB
:10B18100C5A632201003022FC07581D87438C0E0E3
:10B19100E4C0E03212B1B280C6C218B40202D218C1
:10B1A10012BDA630180874E412D46602B0C102B010
:10B1B100BC78A7E66002162230754079AA7700E5CF
:10B1C10079602C14FF760D24CE4006EF90B23B93AC
:10B1D100F6301C1FEF249C7410400BEF240A75F00D
:10B1E100DFA4746F95F0C21CF5B4C313F5B22278D5
:10B1F100A7767DD21CE4F5B4F5B222E57924CE50D0
:10B20100097628301CED741480DC79A1E57997402A
:10B21100E2E57979AAC7272464200E03F4242CFFE0
:10B22100301C06EFF6243680BDEF200D02C313F665
:10B23100EF300D022436D21C80AE78726D68635FE8
:10B241005B57534F4B4845423F3C39373432302DE1
:10B251002B2928262422211F1E1D1B1A19181716F7
:10B26100151413121110100F0E0E0D0DD2B5C28E42
:10B27100AE8DAA8DAF8BAB8BE4F58DF58BD28E3075
:10B2810014012278B6BE0007EF24E24002800806CE
:10B29100E624EC50027614E624F64005E4FEFAFFBB
:10B2A100FB7C007D0A1264697C007D5E1265898FDA
:10B2B1007EEE6003757EFFEAFC7A3312647DEBF566
:07B2C100F0A4E5F0CB8CF0D6
:10B2C800A425E0C5F035E0CB926C25F050060BBB09
:10B2D8000002D26C30E7060BBB0002D26CECF5F032
:10B2E800A42BFBE5F03400FC306C010C78A6E6C317
:10B2F8009BFF18E608F6EB18F618E69CFE18E60819
:10B30800F6EC18F6301401227A0050040A1267008D
:10B318007C007D6E1265898FF078A2E6A4FBACF004
:10B3280012669FEBBA0002F404FAE4F8FFEA30E789
:10B338000118E57960062075031FF4042AF579EFF2
:10B3480038D27520E70860037579FF02BFB0C2756F
:10B358000470F5E579F40460EFF57980EE1216E6ED
:10B36800E5BE78A2F624F65007E4F5BEF6124F982B
:10B378001216E185BC2B85BD21E5BEF54824F650A3
:10B3880008E4F5BEF548124F98E5BFF54324F85098
:10B398003B24F340371216DC78A1E5BCF624CD50E7
:10B3A800087432F5BCF6124F98E5BD24F6502824EF
:10B3B800914024E5BF789DF61424FB50087403F6E9
:02B3C800F5BFCF
:10B3CA00124F9878B7A6BED25322740AF5BFF54336
:0DB3DA00124F9880BE75BD0F124F9880D4A1
:10005E0078FFE4F6D8FDF478D8F6F5A6D220D2B41F
:10006E00D2C075C07A75D75075AE1375AF01758154
:10007E00D875A882D2BC758951D28C7590F875EF5F
:10008E00BC75FDFFC258D25912B365D2A412D3E18A
:10009E00C2A412B3E712D48D12BC90C22012CFAFFD
:1000AE00C22B122E007F527E0090966A1273181287
:1000BE004E9912D30F12D3E1745012B1E712D3E15D
:1000CE0012B1F41249F912D16F12D30F12D3DA759D
:1000DE003A00124A1EE53A701612D4C37F437E06CA
:1000EE00909BF912731812D30F12D3D4022FC0752E
:1000FE00A6FF1207B3C22B302B2E122E001208BCF5
:10010E001208E91208047F7B12225512D30F7A3C93
:10011E00D234204405741812B1E712D3E512B1F4AB
:10012E0012D3E5100202DAEA1249F912B365122E61
:10013E000012D30F12D3DDE478B5F6F52012BC858C
:10014E00C215122E009096897F78127300205E0AD7
:10015E007F767E1290969612CA047F4012D2EB7F63
:10016E00497E0E78AEE612C8D97E18743B12C9D6F7
:10017E007E1BE53E12C8D97E25743B12C9D67E2859
:10018E00E53F20E00805A6E5A6700215A6E53F129C
:10019E00C8D97F5312C1AE7F577E0B12C79B12C8B0
:1001AE00237F6030736A7E0BAC5DAB5C12C79F120F
:1001BE00C8237E311273A37F6A7E1212CD057F7221
:0201CE007E00B1
:1001D000E5A612C94212D30F1000531001531002AA
:1001E00053124997D2AC75369612D21EB4E005125E
:1001F0004A64800CE53670F11249E712D3DA801BAD
:10020000302B18E53FA2E0921D12027230740C20D0
:100210002C0978B50606E624E2401602014B20744C
:10022000097E2BE52E540712C9C37E178094022F36
:10023000C0023182020946D215C221909BED7F781F
:100240001273001208BC7F577E0B909D7E127318AC
:100250007F607E08909D861273187F6A7E0D909D48
:1002600091301D03909D9812731802D30F1249D933
:100270008008D232301DF61249C11000B178A9E6CB
:100280007007E532243850282230210312023778D3
:10029000A9E624F6401A7F607E08909DA01273188C
:1002A0007E36E612C9C312D30F64017003752000B5
:1002B000D2AC12D21E301D05B443BF8005B440BA83
:1002C000F53875A6FF78A9E6760C24F64002D2210F
:1002D000201D3412D21EB4693C12D21EE5387008BB
:1002E0001207B3202B05808C0203849006F4E024CF
:1002F00020F012D0D37F0B9006EAE0A312D07FDF6C
:10030000F912D0890202741249C1746312D07F12AB
:10031000D3EB020274B46C2D12D24EFC12D24EFBFF
:1003200012D21EE538705D1203FC4058B44C0280B6
:090330005512D0D37E7C90070029
:10033900E0A312D07FDEF912D0898047B46647D294
:100349003212D24EFC12D24EFB12D24EF51212D2FA
:100359004EFD12D24EF51312D21EF51412D21EF50D
:100369001512D21EE5387013120446400E1249D9EF
:10037900EDB45102C23212D07F8008744F1249D9AC
:1003890012D07F020274B4703612D21EE53870EBB7
:100399002032E812048740E312D0D3747012D07F60
:1003A900ED12D052EC12D052EB12D052EDB4C90A70
:1003B900EB24FEF513EC34FFF51412D08980C4B494
:1003C90067B912D24EFC12D24EFB12D24E1470AB48
:1003D90012D21EE53870A41204BE409FB44C0280AC
:1003E9009C12D0D3900700E0A312D07FDEF912D07F
:1003F90089809012D0CE746C12D07FEC12D052EB5F
:1004090012D05212D0891249C1D2AC12D21EC5F0F3
:100419006029C5F0B44F028022B44C02C322B44013
:100429001AF5387E7D90070012D21EC5F0600CC502
:10043900F0F0A3DEF3E5387002C322D32212D0CE46
:10044900746612D07FEC12D052EB12D052E5121220
:10045900D052ED12D052E51312D052E51412D07FCA
:10046900E51512D07F12D0897E1E1249C1D2AC1275
:0D047900D21EC5F07004DEF78039ADF0C36F
:1004860022787012D0BFD2AC12D21EC5F06027C53A
:10049600F0B44F028020B4401DF53812D21EB4705D
:1004A6001512D24EFD12D24EFC12D24EFB12D21EA5
:1004B600E5387002C322D32212D0CE746712D07FE1
:1004C600EC12D052EB12D052740112D05212D089D3
:1004D6007E06EC65147007EB651370027E141249F4
:1004E600C1D2AC12D21EC5F07004DEF780C8C5F0CA
:1004F600B44F0280C1B44C02C322B440B9F5387E71
:100506000090070012D21EC5F060ABC5F0F0A30E36
:10051600B42AF112D21EC5F0609CE5387098C32249
:100526001249D9744F12D07F80057F40121709D225
:10053600151249D9D2AC10007B12D21EB440F7F581
:100546003812D21EB44BD97E0B9006F512D21EC5B8
:10055600F060CDC5F0F0A3DEF37E0090070012D266
:100566001EC5F060BBC5F0F0A3DEF312D21EE5385F
:1005760070AE1205BD40A912D0D3744B12D07F7E47
:100586000B9006F5E0A312D07FDEF97E00900700FF
:10059600E0A312D07FDEF912D0897F3F7E35909C92
:1005A6006D12731812D30F12D3DAD2A412D3E1C28A
:1005B600A412CFAF020B2712D0CE744B12D07F7E7F
:0905C6000B9006F5E0A312D07FB2
:1005CF00DEF97E00900700E0A312D07FDEF912D093
:1005DF00897E501249C1D2AC12D21EC5F07004DE12
:1005EF00F7803FC5F0B44F028038B44035F538126C
:1005FF00D21EB44B2D7E0B9006F512D21EC5F060A5
:10060F0021C5F0F0A3DEF37E0090070012D21EC5C5
:10061F00F0600FC5F0F0A3DEF312D21EE5387002C2
:10062F00C322D3221249D9744F12D07F80057F5233
:10063F00121709D2151249D9D2AC10004012D21E8E
:10064F00C5F060F6C5F0B440F1F53812D21EB464AF
:10065F00D312D24EFC12D24EFB12D24EFD12D21E2C
:10066F00E53870C012068F40BB12D0D37E8490073E
:10067F0000E0A312D07FDEF912D08980B6020B27DB
:10068F0012D0CE746412D07FEC12D052EB12D05233
:10069F00ED12D05212D0891249C1D2AC12D21EB46F
:1006AF00401AF5387E8590070012D21EC5F0600CF7
:1006BF00C5F0F0A3DEF3E5387002C322D3227F5BCF
:1006CF001217097946784312D0B6D2AC12D21EC592
:1006DF00F0700510001680F4C5F0F54B12D21EF520
:1006EF004CC2AC12518D12D30F12D3D4020B277FF1
:1006FF002E12170912073112073E12D30F100008DE
:10070F0010011210023980F51512E51224CE40E7C0
:10071F0075123280E20512E512243750DA7512C8CD
:10072F0080D5786512D0BFD2AC12D21EF512227FBF
:10073F002D7E3B742512C9D67E28E51202C88B790F
:10074F0045A81212D0B6D2AC7E1412D21EC5F070CC
:10075F0002DEF7C5F0700E7E20909C7A127318128D
:10076F00D30F12D3DAC2AC020B277F3712170978D7
:10077F006D12D0BFD2AC12D21EFC12D21EFBC2AC75
:10078F0012645C1F7E2FE51B12C9C37E35E51A125A
:10079F00C9C37E3BE51912C9C312D30F1002C81289
:1007AF00D3E580C6C22BC244C2437F05786912D0FD
:1007BF00BFD2AC12D21EC5F06023C5F0B44F028079
:1007CF001CB440EF7E0C75A7009006EA12D21EC52E
:1007DF00F0600AC5F0F0A3DEF3E5386004DFCD80EA
:1007EF0011D22B9006F4E0B45302D2446445700248
:1007FF00D243C2AC227F05786A12D0BFD2AC12D2DC
:10080F001EB44018F5387E0D90070012D21EC5F0A9
:10081F00600AC5F0F0A3DEF3E5386005DFD90211F9
:10082F002CC2AC7F757E009006FF7513041251E643
:10083F00D513FA9007077513041251E6D513FA1260
:10084F00D30F02D3DAE53524C85050E59020E24BA0
:10085F00D0E0D0E01208AB026048E53524D2503B1F
:07086F00E59020E236D0E025
:10087600D0E012D4C3020935E53524D25026E590DE
:1008860020E221D0E0D0E012D4C3306B119098E77B
:100896007F0912730012D30F12515C12779212085D
:1008A600AB020A512212D4C3909C7F7F00127300C0
:1008B60012D30F02D3DA7F407E02909D4512731841
:1008C6007F4978037E017512069006EA1209297E91
:1008D60012909D5012731878037E2F75120690069B
:1008E600ED80407F5630430512CC0C800E7E08907A
:1008F6009D56204403909D5F1273187F637E02907D
:100906009D6812731878027E2F7512089006F012F1
:1009160009297F6C7E02909D7312731878027E2FD0
:100926009006F2E012C9D6EE2512FEA3D8F52212E1
:10093600D4C3909C7F7F0012730012D30F12D3DDB5
:10094600C215C214C227C268E4F535F52075370111
:1009560090971E12215690096073020136021C57A9
:100966000213EA022341020A51020A900260480277
:1009760009D9020984020B27020B27020B27100252
:10098600BF1001051000B980F510020D1001B1105D
:10099600000280F5124FA380A7D25312D4C3F54BA1
:1009A600F54C124987E54B12D073054BE54C12D036
:1009B60073154CD2AC7F3C12D21E7E0512C88B1228
:1009C600D21E7E2312C88B12501012D3E53000D2ED
:1009D600020946E4F535F520753707909A6012212D
:0809E600569009EB730209466B
:1009EE00020ACD020AFA020A0C0209D90209D90238
:1009FE004CC8024ECA020A11020A1C0212A2124A64
:100A0E0021801C124E63124F8912CFAF80BD7F52D0
:100A1E00A25E12159A925E1215B580AF124F98E42F
:100A2E00F535F520753702909B7A122156900A3FC4
:100A3E00730209D90217110217760217CD02181187
:100A4E00021855C268E4F535F520753705909863A0
:100A5E00122156900A657302094602755602759B5D
:100A6E00027730020A51020A8902766F0276D502A7
:100A7E001C20020A51021C0602152F7F2E121A810B
:100A8E0080C1E4F535F52075370690992012215670
:100A9E00900AA273020946021C5D021CB7021D28B1
:100AAE00021DF5021E27021E9E020A90020AC302B2
:100ABE001ED1021F767F49121A8180C6124F98E40A
:100ACE00F535F520753703909AB8122156900ADF46
:100ADE00730209D90218DE02155002155B02194085
:100AEE00021BB40219580215C1124F98E4F535F5E0
:100AFE0020753704909B39122156900B0C73020906
:100B0E00D902156A021575021580021B15021B5EAD
:100B1E0002186402186802158F302B33E4F535F590
:100B2E002075370A909DAF122156900B3C73020927
:100B3E0046020B65020D0002113C020B270206FE57
:100B4E000207790205300214B302063D0206CD7F7C
:100B5E00631215E00209461212D650027800881070
:0E0B6E001212D84049120C5E12224212D30F0E
:100B7C00A81010000810010D10021280F518B8FF13
:100B8C00DF780B80DB08B80CD7780080D3A8101264
:100B9C000C5E1222D612D30F12D3DD1000231001DB
:100BAC001210020280F5A810121325500312112CFA
:100BBC00020B2775A7009004007F56745FF0A3DF2B
:100BCC00FCA810120C5E12224212D30F7F0F90045D
:100BDC0000120C1F7F1990040A120C1F7F23900423
:100BEC0014120C1F7F34900420120C1F7F3E9004B3
:100BFC002A120C1F7F4F900438120C1F7F60900438
:100C0C0042120C1B7F71900446120C1F020B997937
:100C1C00048002790A7E0275A700E0F8D224BE0295
:100C2C0002C224C083C082C001128049D001D0828C
:100C3C00D083E8F0102308A3EE2406FED9DC2209A9
:100C4C00E58224FFF582E58334FFF583CE24FACECA
:100C5C0080C812D4C37F017E14909E1912734B7EF0
:100C6C0036E80412C8DF7F087E08909E2212734B70
:100C7C00C0007F0F900400120CED7F1990040A1233
:100C8C000CED7F23900414120CED7F2D7E08909EAA
:100C9C002912734B7F34900420120CED7F3E90048C
:100CAC002A120CED7F487E08909E3612734B7F4FB4
:100CBC00900438120CED7F597E08909E4112734BB4
:0F0CCC007F60900442120CE97F6A7E08909E4A76
:100CDB0012734B7F71900446120CEDD000227804F6
:100CEB008002780A7E0275A700E0A312C9D6CE2433
:100CFB0006CED8F5227520001213605002780088BA
:100D0B001E1213624047120F8D12224212D30FA8EC
:100D1B001E10000810010D10021280F518B8FFDF2D
:100D2B00780B80DB08B80CD7780080D3120F8D12AC
:100D3B0022D612D30F12D3DD100031100112100284
:100D4B000280F5A81E1213AF500312112C020B27B1
:100D5B0075A704900513E4F07E0E7F06E4F0DFFD2B
:100D6B007F0A745FF0DFFDDEF175A700120F4812EA
:100D7B000F8D12224212D30F120E49C22412803B46
:100D8B00900513F07F177E1D12C1A80F7E1D12C197
:100D9B00A87F117E23909DA912731812D30F75A7EC
:100DAB000490050C78AD120E5D120E5D120E5D787F
:100DBB00AD10000810010A10022380F3124BF380D0
:100DCB0003124C0A75A70490050C78AD120E6C1229
:100DDB000E6C120E6C120F8D12224280A7120F8D09
:100DEB00741A7F1B120E7B120F8D742A7F22120E28
:100DFB007BE5116024751001C010120F8DD010E52A
:100E0B001075F007A42423FFE510C4244A120E7BAF
:100E1B000510C3E511951050DF120F8DE51175F01C
:0D0E2B0007A4242BFF743A120E7B120F8DCA
:100E3800E51175F007A42432FF744A120E7B020DE7
:100E4800377F017E3A900513E0F51124F6E050044F
:100E5800E4F0F51122E0540F75F00AA4F9E0540FFC
:100E680029F61822E675F00A844430F0E5F044309B
:100E7800F01822751400F5138F127E10780875A7E4
:100E880000758305851382AF12E0A312C9D6CE245C
:100E980006CED8F512225212D30F100008100127DF
:100EA80010024780F57E01E53524DC50027E0415EA
:100EB80014E514B4FF037514DF120EF3E56FB4FFE5
:100EC8000280ECDEEA80B37E01E53524DC50027E48
:100ED800040514E51424205003751400120EF3E5DC
:100EE8006FB4FF0280EBDEE9809022E51475F00410
:100EF8008424A8F5C675C70375B901A9BCE5F060D7
:100F08000CA9BD146007A9BE146002A9BF89158980
:100F18006F127A70758305E51324FAF582E566F099
:100F2800A3E565F0A3E564F0A3E569F0A3E568F03F
:100F3800A3E567F0A378D07F07E6F008A3DFFA22DD
:0D0F4800C01E124A42124A42D01E75A70474
:100F5500900500120F74E53D120F80E53E120F80DB
:100F6500E53F120F80120F747401F075A70022E59A
:100F75003C120F80E53B120F80E53A75F00A844478
:100F850030F0E5F04430F02212D4C37F017E0190A9
:100F95009F9B1273187E1AE51E0412C8DF7E2C90E3
:100FA5009FA8127318120E4912C9C375A70490059C
:100FB500007F0A1210BD7E27E012C9A47E2BE01225
:100FC500C9A47E2E743A12C9A47E31E012C9A47E4A
:100FD50035E012C9A47F1190050C1210BD75A7004C
:100FE5007E23909FA012734B7F1912C1A67F1C9080
:100FF5009FAB1273499005141211057F238F17902B
:101005009FAF12734990052412110512BFEEE4F546
:101015001CF51BF56EF56D126D18E511603E75102A
:1010250001E51075F007A42424FFF517909FA81279
:1010350073497E08E51012C991C42444F58275836D
:1010450005121105126D8D2032031210EF12BFEE3D
:10105500126D180510C3E511951050C5E51175F011
:1010650007A4242CFFF517909FB3127349900534FC
:10107500121105126D8D2032031210EF126D18E555
:101085001175F007A42433FFF517909FB712734924
:10109500900544121105AE6EAF6D7C007D0512659D
:0F10A50089126D6FAC06AB071264537F717E1812
:1010B40012C7A20F7E370295F27E00E012C9A47E09
:1010C40004E012C9A47E08742E12C9A47E0CE01296
:1010D400C9A47E10E012C9A47E14742E12C9A47E81
:1010E40018E012C9A47E1CE002C9A4AE1CAF1B7C8C
:1010F400007D0A126589E56D2FF56DE56E3EF56E8E
:101104002275A704E0F566E0F565E0F564E0F569AD
:10111400E0F568E0F5677E107807E012C9A4CE24F4
:1011240004CED8F675A700227F797E17909C7012A2
:10113400731812D30F02D3DAE4F535F520753708A6
:10114400909E7B12215690114E73020B2702115D63
:101154000211820211A80211D47F0A121709121A6D
:10116400C710000810010D10024D80F5E51260EE65
:10117400151280EAE51224F640E4051280E07F139C
:10118400121709121AC710000810010E1002288045
:10119400F5E5131460ED151380E9E51324FC40E331
:1011A400051380DF7F1C121709121AC710000E10D6
:1011B400011410020280F512123502113CE51414D8
:1011C40060E7151480E3E51424EC40DD051480D9B0
:1011D4007F25121709121AC7100008100105100202
:1011E400D680F5E515B45904744E80027459F5158A
:0611F40080E37F0A78751C
:1011FA0012D0BFD2AC12D21EC5F06025C5F0B440E1
:10120A0020F53812D24EF51212D24EF51412D24EE1
:10121A00F51312D21EF51512D21E12D21EE538602F
:10122A0006DFCBC2ACD322C2ACC3227F0512D0CE1A
:10123A00745512D07FE51212D052E51412D052E53D
:10124A001312D052E51512D07F12D07F12D0891214
:10125A0049C1D2AC12D219C2ACC5F07004DFCE803B
:10126A00C2C5F0FDB451F680BEE51224F5500375EF
:10127A001200E51324EB50067404F513F514E51473
:10128A0024EB50067404F513F514E515B45901223C
:10129A00B44E012275154E22E4F535F520F5379046
:1012AA009E561221569012B3730209D90212C20233
:1012BA0012C70212CC0212D11250AE80DB12502099
:1012CA0080D6124FA380D1124CCE80CC783F7F0AB1
:1012DA00796812D0B6D2AC12D21EC5F06033C5F00E
:1012EA00B44F02802CB44029F53812D21EB46821BA
:1012FA0012D21EF824F440197E5775A700900400F4
:10130A0012D21EC5F0600AC5F0F0A3DEF3E538601C
:10131A0006DFBDC2ACD322C2ACC3227F0512D0CE37
:10132A00744812D07FE812D07F75A7009004007E1F
:0D133A0056E0A312D07FDEF912D0897E1E8E
:101347001249C1D2AC12D21EC5F07006DEF7DFD04B
:1013570080C4C5F0B451F780C1783F7F0A79741211
:10136700D0B6D2AC12D21EC5F06033C5F0B44F026E
:10137700802CB44029F53812D21EB4742112D21E23
:10138700F824F440197EE575A70090050012D21ED7
:10139700C5F0600AC5F0F0A3DEF3E5386006DFBDEF
:1013A700C2ACD322C2ACC3227F0512D0CE74541272
:1013B700D07FE812D07F75A7009005007EE4E0A3F8
:1013C70012D07FDEF912D0897E1E1249C1D2AC122B
:1013D700D21EC5F07006DEF7DFD080C4C5F0B45169
:1013E700F780C1D25712D4C31222421213F802094E
:1013F700467F177E0290978E1273187F4C7E02905D
:101407009799127318AC5DAB5C7F577E0412C81BAB
:101417001216F585BC6285BD637F377E0F74461251
:10142700C9D67E15744C12C9D6E560240FFBE43586
:1014370061FCA25C923BD25C7F377E1E12C79FA2E3
:101447003B925C7E30742012C9D67E36742012C956
:10145700D6E5602562FBE5613563FC7F227E0412D9
:10146700C81BE56245637015742E7E3A12C9D61201
:10147700D30F10000C100114100225809C742080DB
:0C148700E91562E562B4FF0C15638008F3
:101493000562E56270020563E53524F55003753393
:1014A300010214201216F58562BC8563BD024F98B4
:1014B300C214C21512D4C31222421214C3020B2740
:1014C3007F177E02909FBB1273187F377E02909F17
:1014D300C61273181216EB85BC6285BD63AC63AB91
:1014E300627F227E0412C81BAB60AC617F427E0424
:1014F30012C81B12D30F10000810011010022C8009
:10150300DC1562E562B4FF0C156380080562E562D1
:1015130070020563E53524F550037533011216EBAC
:101523008562BC8563BD124F9880B2221222AB1232
:10153300D30F10001510010280F87F637E05909889
:10154300E712731812D30F12512B020A517F13A201
:101553000D12159A920D80097F1CA20E12159A92F4
:101563000E1215B5020ACD7F0AA20812159A920827
:1015730080147F13A20B12159A920B80097F1CA271
:101583000912159A92091215B5020AFA7F49A20F98
:1015930012159A920F80EF8F1F92171217091216C6
:1015A300E185BC2B85BD21AF1F1F7E39127FE6A2CB
:1015B30017221216E1852BBC8521BD024F982037D7
:1015C300141216DC85BE121215EE1216DC8512BE3D
:1015D300124F9880057F3F1215E0020ACD7E0390DB
:1015E3009B0112731812D30F02D3DA75A6FF12D41C
:1015F300C3C22F740712D4AF8FF0740612D4AF1086
:031603002FEFEFD7
:101606002512C395F0FD78D8E6C4540F2DA2E792B3
:101616003D4010FD24CD50027D32AC05C3743F9D84
:10162600FD800FF404FD24C850027D37AC057440DC
:101636002DFD7F4012C1A67E1212D4060EBE1EF9E3
:101646001F303D020F0FEF6D70EDE536700A7536EF
:1016560006EC2513F5148C1312167712D30F10000F
:101666000710010830020722151280020512021522
:10167600EE7F377E28742E12C9D67F347E21740AF7
:10168600303D010412C9F3E514FC249C50027C632E
:10169600EC75F00A84C0F07F347E2D12C9F3D0E0D9
:1016A6007F377E3612C9C37F437E1E12C79B7E00DC
:1016B600E51212C9327F057E02909B0D1273187FC8
:1016C6006D7E01909B1812734B7F747E04909B2A4B
:1016D60012734B02224275C6F8802175C6F9801C2A
:1016E60075C6FA801775C6FB801275C6FC800D7527
:1016F600C6FE800875C6FF800375C6FD75C70375EF
:10170600B90122743F12C9A402D30F7F0A12170926
:101716007E2A124A211216E6A8BF12174510001299
:1017260010010510021580F508E824E750EC78183A
:0B17360080E818E830E7E3780080DF6F
:1017410088BF80627F097E05909DA9B80C03909C9B
:10175100E01273187E27E53D28240C75F01884E506
:10176100F012C86E7E33743B12C9D67E35E53E1247
:10177100C86E02D30F7F131217091216E185BC2B15
:101781001217AA10000810010510021780F2105C50
:1017910007205D0BD25C80E8105DE5D25D80E1D26F
:1017A1005C80DD852BBC020A2A205C10205D18902C
:1017B1009EAD7F127E2312731802D30F909EC1201B
:1017C1005DF0909EB480EB909EBA80E67F1C12176C
:1017D100091216E1A8BF1218041000081001111017
:1017E100021A80F2E824F750031880EA780880E6AC
:1017F100E824EC40030880DE781480DAE8F5BFF5D0
:101801004380A37F1B7E2EE8232312C87402D30FCB
:101811007F251217091216F0A8BCE812184C12D332
:101821000F10000810010D10021F80EEE824E05097
:10183100E9188006E824CF40E1081216F088BC12AE
:101841004F98D21512CFAF80D180157F247E3724D7
:10185100E202C8DF7F2EA20A12159A920A1215B56A
:10186100020A2DD23D8002C23D7F40303D027F37CA
:101871001217091216E6A8BD303D02A8BC1218A81D
:1018810010000810010D10021280F218B8FFEE7856
:091891007D80EA08B87EE67800CB
:10189A0080E2203D0488BD800288BC020AF77F3FAF
:1018AA00303D027F36E82312C54D75F06484C0F0DE
:1018BA007E2012C9C37E26742C12C9D6D0E07E2996
:1018CA0012C86E7E35909EC7305D03909ECA127311
:1018DA001802D30F7F0A1217091216DCA8BCE812E5
:1018EA00191212D30F10001010010510021280EE07
:1018FA0018B8FFEA783280E608B833E2780080DE6A
:10190A00E8F5BC79A1F78072305C01237F097E2358
:10191A0075F00A84C0F012C8DF7E2D742C12C9D665
:10192A00D0E07E2F12C9BC0F7E35909ECD305C036D
:10193A00909F2902734B7F251217091216E6E5BEFE
:10194A007F247E2C12803BF5BE79A2F7802C7F374C
:10195A001217091216E1E5BC20E201E4540375F0FE
:10196A0003A47F367E3212803B0475F00384600242
:10197A002404F8E5BC54F848F5BC020ACA1216E178
:10198A00E5BE7F097E3A02C9C31216E6A8BF12173E
:10199A00451216E185BC2B85BD211217AAA8BF12D4
:1019AA0018041216F0E5BC12184C7F2DA20A021A6E
:1019BA003A1216E185BC2B85BD217F12A20D121A9F
:1019CA003A7F1BA20E121A3A1216DCE5BC12191241
:1019DA00A8BF121BF2E52B540375F003A47F367ED1
:0919EA003212C9C31216E6E5BE73
:1019F3007F247E2C02C9C31216E6A8BCD23D12185E
:101A0300A8A8BDC23D1218A81216DCE5BD121B46DC
:101A13001216F0E5BD121B8A1216E185BD217F095E
:101A2300A208121A3A7F12A20B121A3A7F1BA209BA
:101A3300121A3A7F48A20F744E400274597E3A023A
:101A4300C9D61216E185BC2B7F51A25E80E91279BB
:101A5300867F7312761C1279D57F6C12762B7F2DBD
:101A6300800E1216E1E5BE7F097E3A12C9C37F4894
:101A73007E1E9098FB30530390990002731812173F
:101A8300091F121A7312D30F100008100105100258
:101A93000980EF1053ECD25380E8221262F6EBF583
:101AA30016F5147F6C12762B1262DA7F647E23E5BF
:101AB3001612C942C3E5169514F5167F7312761CE8
:101AC3007F2480ACE51224F5500375120AE51270E9
:101AD30003851413C3E51495135003851413E512FA
:101AE3006009E51324FB50037513047F097E2CE57D
:101AF3001212C8747F127E2CE51312C8747F1B7EEA
:101B03002CE51412C8747F247E37E51512C9D6025A
:101B1300D30F7F251217091216DCA8BDE8121B4646
:101B230012D30F10000810010D10021280EE18B826
:101B330009EA787880E608B879E2780A80DE88BD19
:0D1B4300020AF77F247E2975F00284C0F0AD
:101B500012C874D0E075F005A47E3B02C9C37F2E85
:101B60001217091216F0A8BDE8121B8A12D30F1023
:101B7000000810010910020D80EE18B8FFEA08B83D
:101B8000C9E61880E388BD020AF712C54D7F2D7E95
:101B90002675F00A84C0F012C8747E32742C12C903
:101BA000D6D0E07E3512C9C37E3B7422305D02740C
:101BB0006602C9D67F2E1217091216DCA8BFE824C8
:101BC000FA40033037027803121BF212D30F1000D1
:101BD0000810010D10021280E518B800E1780580A8
:101BE000DD08B806D9780180D5799DE8F7F5BF0200
:101BF0000ACA7F2D7E2C7420B80502742E12C9D615
:101C00007E32E802C9C3D26875480A124A21D2144A
:101C1000122FF8127AC01239E1C26B12087E80F3DB
:101C2000D21475150112794075B901E5BC20E71C85
:101C3000127A7075A6FF127ACC12226812D30F1294
:101C4000742010000F500512754880E70515E51542
:101C5000242050D1020A51121C63020946121C634F
:101C6000020A90121C6F1216E18548BE024F9812AC
:101C70002FEA123004126B0712D4C3909983128D8D
:101C8000E6128D9E12221812D30F100014100105B7
:101C900010021B80F50548E548640A7002F548808B
:101CA000D11548E54864FF700375480980C485482C
:0D1CB00049123004E55822122FEA854849F8
:101CBD00C250E558B40F02D250126B078038D227AC
:101CCD0075480A122FF8126B0712D4C3128CFC90B0
:101CDD009C41202903909C4C1222CCC26A1239E1FE
:101CED00106A0280E1C227127918854948122085B1
:101CFD00123004126B0712D4C3128DE320500E1252
:101D0D0022B612D30F1000101001B380F812226802
:101D1D0012D30F10000280FB020A90122FEAE55831
:101D2D0030E7137F1B909C2B7E0512731812D30F77
:101D3D0012D3DD020A90123004126B078559491235
:101D4D00D4C3122252909C4C128DE6128DA812D340
:101D5D000F10000810010A10020C80F5121DC08032
:101D6D00DB121DCD80D612D4C3122252909993123C
:101D7D008DE6128DA8128DAC12D30F100008100134
:101D8D000A10020C80F5121DD980DB121DE780D6DA
:101D9D0012204B123004126B0712D4C3909BBF124A
:101DAD008DE612229012D30F10000510028880F8D4
:101DBD00020A900559C3E5589559500375590022EB
:101DCD001559E55964FF7003855859220549D3E526
:101DDD00491495584003754900221549E54964FF9A
:101DED007005855849054922122FEAE55830E70557
:101DFD007F24021D32123004126B0712D4C3909946
:101E0D009E128DE61222C112D30F10000A1001028C
:101E1D0080F81220F480DE020A90122FEAE5583085
:101E2D00E7057F2D021D32C26B7559FF126B07122C
:071E3D00D4C3122242E55953
:101E440030E70312225D9099AF128DE6128DB8121D
:101E5400D30FE55820E70610000810011110021BEB
:101E640080F00559C3955950CF7559FF80CA15594B
:101E7400E55964FE70C285585980BDE55920E711C3
:101E8400D26B75A700758307C4F582E0B2E7F080D2
:101E9400A7306B031220A2020A90122FEAE55830F1
:101EA400E7057F36021D32123004126B0712D4C3C9
:101EB4009099BA128DE61222AB12D30F10000B10B8
:101EC400010280F81220E912211E020A90122FEA60
:101ED400E55820E7087F519099C4021D3512D4C3F8
:101EE400909C57128DE612226812D30F124987D2A2
:101EF400AC10001FE55830E7F8306DF5121FFA7E7C
:101F0400207F005013909C7012734B12D30F12D386
:101F1400DD80CAC2AC020A901B8B139098E712733F
:101F24004B12D30FC26B7B007514B81220DE127AE9
:101F34003F1279F15025A814E824384004A601057D
:101F4400140BC3E5139B50E678B8122120306B03C1
:101F5400127792123004126B078082127986E5168A
:101F640060E6D26B127A9CC003127957D003A9158C
:101F740080C4122FEAE55830E7057F5A021D321259
:101F84003004126B0712D4C39099CF128DE612223B
:101F94008512D30F10002410010280F8121FC29082
:101FA4009C625003909C70128DE67F007E3CE54B52
:091FB40012C99112D30F12D3DD02
:101FBD0080C4020A9012498712D0A5745212D0D84B
:101FCD00745412D073E5580475590012D0941273DD
:101FDD00D04016127918127A70127420400B0559E0
:101FED00C3E558955950ECC322C2ACD32212498790
:101FFD00D2AC12D219C5F060F0C5F0B440F412D2D3
:10200D001EB4400312D21EB452DFF53812D21EB4E4
:10201D0054D712D21EFA60D124EF40CD12D21EE554
:10202D003870C612D21E12D21E1273B57B001274F6
:10203D00A840B6127A4F0B1273B5DAF2C3221221F1
:10204D002FE55924C8F88602E54924C8F99860138C
:10205D00146010500F18E608F618E86970F7A7021B
:10206D0012211E22E559640F60F91908E618F608C9
:10207D00E86970F7A70280E812212F78C8C250E6F0
:10208D00B4FF02800708B8D8F6D25022B8D702D2D2
:10209D0050A615807C78B8122131E4F9F5A7758327
:1020AD0007E9C4F582E030E70AE924B8F82438409E
:1020BD000276FF09C3E5589950E71220E978B879FF
:1020CD00C8E6B4FF028002F70908E8243850F28010
:0320DD004079B88F
:1020E00077FF09E9243850F82279C877FF09E924F5
:1020F0002850F82212212FC23D78D7B6FF04A9003C
:10210000D23D18B8C7F5203D0279D81978C8B6FF76
:102110000122C3E8995007C6C7C6081980F478C8D9
:10212000122140127AAE127AAE127AAE027AAE78EC
:10213000C8122140127A8A127A8A127A8A027A8A1C
:1021400075C703E54875F004A42480F5C62212D4AF
:10215000C3127304800612D4C3127308E537605C9F
:1021600014605614604E14604614603E14603614B9
:10217000602E14600B14600D14601814601A803CFB
:10218000121A4580371211F6121273121235121AF2
:10219000C7802C121A9E802412073112073E801C21
:1021A000121A658017121A5180121219FA800D1234
:1021B00019BB8008121993800312198712D30F12CA
:1021C000D3E1122242D234E4F5B4F5B2A81F08E8F4
:1021D00014C23BB51D02D23B75F007203C0375F0DD
:1021E00009A4FF203C010F7E007420303B02743EA6
:1021F00012C9A4D8DA12D30FE51D10000810010D82
:1022000010021080C0651F60BC051D80B860B61547
:082210001D80B275F003A42249
:102218007F7B7E00909F8112734BE54824F640082F
:102228007E0A909C0D12734B221276487E05745BD1
:1022380012C9A07E1D745C02C9A01222317E34909E
:102248009F9202734B12764880031222317E31909E
:102258009F9602734B1222317E31909C8002734B01
:102268001276487E0080051276487E2D909C80026A
:10227800734B1222857E3190990502734B122268A6
:102288007E1A90990A02734B12226880C012226843
:102298007E189098D402734B1222687E1A909C85FF
:1022A80002734B1222687E1A909C8A02734B122288
:1022B800687E1A90998D02734B1222687E18909945
:1022C800A902734B7F007E2012734B02D30F127644
:1022D80048909C9002734912B67E1216FFE5BDF530
:1022E8005EF56CE5BCF55FF56B756A007561FF75A9
:1022F800A70490070012B62AB4FC12E582C313F5AE
:1023080061E56CF0E56BF0E58260168005B4FF02CC
:10231800800F12B570E56C655E70DAE56B655F700D
:10232800D475A70022E560758307C333F582E0A35F
:10233800F56CE0F56B756A0022D214C21F1222DF19
:10234800756000E561B4FF1612D4C39097BB7F0A8D
:102358007E0512734B12D30F12D3DA020946C2104C
:10236800C21112D4C3122242301F0A7F079097C9A4
:0A23780012734980647F007E01C3E8
:10238200E56012C9427E0E742812C9A085604874A5
:1023920007F51FFF7E00743E12C9A4E54812232FE1
:1023A20012BFCC1228B50548C3E5619548FD401C13
:1023B200E51F2407F51F24C850E17F387E01ED0494
:1023C20012C9427E0E742912C9A0800DE51F24078E
:1023D200FF7E01909C7F12734B201F031228F8127C
:1023E200D30F10001910012C10020280F512086997
:1023F200301F3D020935101F02D21F022366E5611C
:1024020060F4E56065617005201FF080E9201FE639
:10241200056080E7E56160DEE56065617005201FAB
:10242200D58009201FD5E560700280CA156080CB77
:102432001222DF12232D12BFCC1229EC756A101260
:10244200B611122AA39097D01273041221C29024BB
:10245200547302236602382C02247D022460122265
:10246200AB12D30F1000C910010280F812232D12F3
:10247200B62AC2E2FF12B4B1022341C25312232D83
:1024820012BFCC7537009097E912215690249273AF
:1024920002243202267F02268402247D0224B9020B
:1024A20024BE02247D0224FC02250002250402250A
:1024B2000B02250F0225131249B4800312499F789B
:1024C2000A1225DC740512D07112261B12D08D124D
:1024D200265612B61112B63D12B52E12B754122755
:1024E2006CD5150C75150A12266912287F12D08D2B
:0A24F200100204E57F70DB022432C3
:1024FC00780A80067804800278011249B4800D783D
:10250C000A800678048002780112499F1225DC7437
:10251C000512D06612261BE54812D052742A12D02E
:10252C007312D07312D07312D08D12265612B611AC
:10253C0012B63D12B52E12B75412276CD51548851C
:10254C004815122669E51C12D052E51B12D052E533
:10255C001B2548F51BE4351CF51CE4A27792E7A279
:10256C007492E0A27392E112D052AD75AC74AB735D
:10257C00E57DC412259DAD78AC77AB76E57D122553
:10258C009D12289D12D08D100204E57F709F0224AD
:10259C0032540F2375F00584F8C3EB33FBEC33FC9A
:1025AC00ED33FDC3EB33FBEC33FCED33FD20E713D4
:1025BC00EB28FBE43CFCE43D12D052EC12D052EB85
:1025CC0002D052C3EB98FBEC9400FCED940080E835
:1025DC00884812226FE4F54AF549756A2075150191
:1025EC0012B61112B52ED5150E854815E5492401E4
:1025FC00F549E4354AF54AE57F70E5744012D0D8C8
:10260C00747812D073746312D073741702D066127C
:0F261C00285AE56012D05212232D12BFCCE53A96
:10262B0012D066E53B12D066E53C12D066E53D1252
:10263B00D066E53E12D066E53F12D066740112D02B
:10264B0052E54A12D052E54902D05212232D756A37
:10265B0020E4F51CF51BF514F513751501227538DF
:10266B0000E51412D052E51312D0520513E5137086
:10267B00020514221249B4800312498A12226F12E6
:10268B0027B512D3E5756A2075150175A6FF754A36
:10269B000112B5B712B52E12B75412276CD5150906
:1026AB0075151E12279012D3EB12287FE57912D0E5
:1026BB0052E57EC333500274FF12D052E5711227DC
:1026CB005112D052E57012D052E57B24ACFFE55F7E
:1026DB00340912D058EF12D052E51520E033857D26
:1026EB0056E412D052E52EC412D05812D09C12D3FD
:1026FB00EB10021A305594744012D073744512D0FB
:10270B0073744F12D073744612D07312D09C022480
:10271B0032E55612272BC4FAE57D12272B2A80C2ED
:10272B00FBC41227382323CB1227382B22540FFC40
:10273B0024F650027C00902747EC93220000010105
:10274B00010202030303FA2440400A24804003EAF7
:10275B003322D2E72274FF2220E703C3132224C0C3
:10276B0022E53F701F7F7B7E0078AEE612C92CEE10
:10277B002404FE743A12C9A4EE2404FEE53E12C9E9
:10278B002612D30F2278AEE612D066E53E12D06643
:10279B00E53F12D066E412D052E412D052740A1202
:1027AB00D05274C012D05202D09C744012D07374A9
:1027BB005412D0D8744E12D073E412D05212285A3D
:1027CB00741712D066E53D12D066E56012D0521236
:1027DB00232D12BFCC78ABE60812D066E60812D0D8
:1027EB0066E60812D066E612D066E53E12D0661297
:1027FB002DE7E51212D066E51112D066740112D0E6
:10280B0052909CA11228A7756A1012B611057F056C
:10281B007F787F12D04B787B12D04B787D12D04BC8
:10282B00787712D04BE4FEFF780712D04B12D04BC7
:10283B00E57412D052E57512D052E412D052E57302
:10284B00C333500274FF12D05212D04B02D09C757E
:10285B00C70375C6FF75B901C217751D0085BC1C72
:10286B0085BD1B85BE1A85BF19126403EE12D052AB
:10287B00EF02D052E57512D052E57412D052E573C7
:10288B0012D052E57812D052E57712D052E576127B
:10289B00D052E55E12D052E57A02D05275A700E411
:1028AB0093700122A312D07380F5AF1F7E0478AD15
:1028BB00E612C9267E0C742C12C9A47E0E18E612E1
:0428CB00C9267E1A82
:1028CF0078AEE612C9267E22743B12C9A47E24E597
:1028DF003E12C9267E2FE54012C92C7E37743B125B
:1028EF00C9A40E0EE54102C92675320012232D121E
:1028FF00BFCC857946787A796412BFE57464126724
:10290F00DE8E471229EC756A20D23D12B61112B62F
:10291F003D122A23303D09307406C23D8E1E8F1F93
:10292F00E57F602BE54C24FFF54CE54D34FFF54D6D
:10293F00454C600512B54680D2751D3C12B611127A
:10294F00B63D12B52E122A23E57F6003D51DED1279
:10295F002A84902A9C12CA04203D0DAE1EAF1F126E
:10296F002A84902A9512CA04E546FD700B909F5158
:10297F00305D11909F4D800C047010909F4D305D15
:10298F0003909F497F38124486804BE4FFFC7E05FD
:10299F00305D047E027FB3126589AC06AB0712640B
:1029AF00537F38C23DE51C6007D23D7E2C12C99182
:1029BF00E51B203D026007D23D7E3012C991E51A1A
:1029CF00203D026007D23D7E3412C991E5197E3851
:1029DF0012C99112448BE53224C850FA22E5407592
:1029EF00F03CA42541FFF54CE435F0FEF54D7C009D
:1029FF007D101265960F8F4BAF4CAE4D7C007D3C1A
:102A0F001264697C00AD4B126596EE4F70010F8F0B
:012A1F004C6A
:102A20008E4D2278647973C2D1122A3AFF78677981
:102A300076D2D1122A3AFE02D406C3E796FB0809E1
:102A4000E796FC0809E796FDA2E792175003126784
:102A50001875135A30D10E751320B217AA47126495
:102A60009DAB04AC05E546600B04600BAA461264FE
:102A7000B4EB03FBEB03FBEB543FFBE5132B2017FD
:102A8000029B9B22EE141430E701E4FEEF14143095
:102A9000E701E4FF2205057088A88870050520205D
:102AA000F8202075320012D4C37E1E7F1C12D4067B
:102AB000DFFB12D4067E1E7F1C12D406DEFB7E1DB9
:102AC0007F1D12D406DEFB7F007E2178ADE612C9A1
:102AD000267E29742E12C9A47E2D18E612C9267EE0
:102AE00035742E12C9A47E3918E612C9267F077ED6
:102AF00021745412C9A47E25744F12C9A47E2D7866
:102B0000AEE612C9267E35743A12C9A47E39E53E76
:102B100012C92678AE122DE77F0E7E21744C12C9A1
:102B2000A47E25744112C9A47E2DE51212C9267E09
:102B300035743A12C9A47E39E51112C9267F157E73
:0F2B400025744412C9A47E2DE54012C92C7E35A0
:102B4F00743A12C9A47E39E54112C9267F1C7E2F23
:102B5F0085715412C6187F217E01909F1C12734BF2
:102B6F007E0EAC77AB7612C7D87E2B85795F8578D2
:102B7F007B12CD5E7F287E01909F2012734B751DB7
:102B8F002B751E10E574122D9B7E25742F12C9A470
:102B9F00751D2D751E2BE575122D9B7F2F7E0290B7
:102BAF009F1412734BE5736003122C487F367E021D
:102BBF00909F0C12734BE572122C48122CE01223CB
:102BCF002D756A209004E6E56CF09004E7E56BF054
:102BDF00AE4DAF4C7C007D40126596BF00010F0FCC
:102BEF00AC07AD07E4FED23D12B61112B63D122C62
:102BFF0089E57F602CE54C24FFF54CE54D34FFF55E
:102C0F004D454C600512B54680DE751D3C0E12B663
:102C1F001112B63D122C8EE57F600612B52ED51D12
:102C2F00ED122C5E7F7812C1B87F767E0074301261
:102C3F00C9A4E53224C850FA227E2112C54D12C90B
:102C4F00427E2F909F24305D03909F2902734B90FB
:102C5F0004E6E0FD9004E7E0FCC3E56A9420FBE5A1
:102C6F006B9CFCE56C9DFD50032410FD1266889053
:102C7F0004E8EEF09004E9EFF022DD03AD040E7FDF
:0C2C8F0078E55E20E72AE57A8549F0A48C
:102C9B00A9F0E57A854AF0A429F9E435F0FAE55E66
:102CAB008549F0A429E435F02AFAE55E854AF0A4BB
:102CBB002ACF9FFF12D406103D18C3EF9B50131B56
:102CCB00EF6B600E8F018B0712D4061FEF6970F844
:102CDB00AF01AB0722909ED1305C03909EEA754A00
:102CEB0040754900AF76E577FE20E76B7005EF2462
:102CFB00105064EF24A8EE34FD4011909ED6305C4A
:102D0B0003909EEE754A1975499A8075EF2450EE23
:102D1B0034FB4011909EDB305C03909EF3754A0CA4
:102D2B007549CD805CEF24A0EE34F64011909EDE09
:102D3B00305C03909EF8754A067549668043EF2414
:102D4B00F0EE34F14013909EE1305C03909EFD75E4
:102D5B004A04754944802A8028EF2490EE34E840D9
:102D6B0011909EE4305C03909F02754A0275498F67
:102D7B00800F909EE7305C03909F07754A01754961
:102D8B009A7F401273497F4612C1B87F5F02C1B868
:102D9B00AE1E75F064305C0375F03284C0F0F870D1
:102DAB0004EE2404FEE51D12C9A4EE2404FEE86023
:102DBB000712C991EE2404FED0E075F00A305C03D3
:032DCB0075F0059B
:102DCE0084A8F012C991EE2404FE742C12C9A40E2C
:102DDE000EE8305C012302C991E53E2541F5112430
:102DEE00C45003F511D3E63540F51224E85002F530
:102DFE001222D23412B1F4C21012D4C37F057E094E
:102E0E009096611273187F137E08902E5212CA0488
:102E1E00302B1E7F2A7E03902F2C12CA04203710CF
:102E2E007F267E14E53F20E0010E902FAC12CA04DF
:102E3E00227F2B7E01902EBA12CA042037F27F27F2
:102E4E007E2980E0113007FE1FE001E101F80F003E
:102E5E00061B00F80C00180E007C10007006003CDB
:102E6E002000E006003E4001E004001E8003C00486
:102E7E00001F0003C004000F00078000000F800732
:102E8E0080000017800F00000027C00F00000043D5
:102E9E00C00F00100083E00F00200301F00700C0F8
:102EAE000F01F80383007F87FE01FC000E3E180021
:102EBE0000030000000018000003000000003800AE
:102ECE000000000000003000000000000000FC7652
:102EDE001F0E1C6030ECFCBC3F172DF0F9786138EA
:102EEE0066264F619A706070C60E1EE330E0606019
:102EFE00C60C1CC360C0E0618C0C18C7C0C0C0E11A
:102F0E008C1C39C611C0C4C19C9931963180C8C180
:102F1E00FF1E31E7E180F0C0EE1C31C38180123715
:102F2E0000000000000E0600000000001806000061
:102F3E000000003000000000000030001DC07607C9
:102F4E0080FC1C2F60BC0CC1F82E4E6138186060DE
:102F5E004C1C60703060601C18E06030C0E01818C7
:102F6E00C06070C0C01838C0E060C0C03839C0C082
:102F7E006180C0323980C07301C03C3700C03E0151
:102F8E0080387000000001800060000000018000A9
:102F9E0060000000030000F00000000E00000616A6
:102FAE003091882892884924904927909248A0E32E
:102FBE00C8BCC2AF74FE12B1E77F6412D3EDC2B4C7
:102FCE0080FC75C703E54875F004A42480F5C6C2DD
:102FDE003C75B901E5BC047002D23C221216E1E543
:102FEE00BEF54824F6500375480075340075370356
:102FFE00C228D229D22A75C703E54824E7500375A3
:10300E004800E54875F004A42480F5C675160775CA
:10301E001700C23C12304512304512304512304571
:10302E008517581558755900E548B40A09E55860D2
:10303E0005F46002055922203C1D75B90105C6AA8A
:10304E00BCABBDACBEADBFEA123066EB123066EC67
:10305E00123066ED12306622203C07F515B4FF03E0
:10306E00D23C22C0C7C0C612794075A7048516830C
:04307E00E517C4F896
:10308200F58275B90105C6E5BCF0C582F82406F9DA
:103092002403C582E5BDF0E5BEF0E5BFF075B901D8
:1030A20005C6E5BCF0E5BDF0E5BFF0851683898273
:1030B200E4F075B90105C685BC1385BD14E4F0F0D2
:1030C2008882E5BEF0E5BFF075B901E5BCF0E5BD6B
:1030D200F0E5BEF0E5BFF0758306E51723541E2424
:1030E200B0F582E513F0E514F075A700D0C6D0C79D
:1030F20005172212B36578BEA64808E4F6F559080A
:10310200761808F6C249C23608760A08F606087624
:10311200BEC225C254C25512B693122FF8C229C29A
:103122002AC227C268C243C24AE4F537F52EF534F3
:10313200F536F52F78A8F678AAF678B6F678B5F6C9
:10314200789EF678B8A65E08A67AC233C238C24024
:10315200C223C222D24175460178C5A646C23AD2DE
:1031620021C219C226C23485705778BA7401F60892
:10317200F608F608F6E4F542F541F540220201367A
:0B318200302B3F1212D64018120C5EDA
:10318D0012229012D30F78B5761E1000E5100205AD
:10319D0078B5B600F5121360401D881E120F8D1202
:1031AD00229012D30F12D3DDC20278B5761E100015
:1031BD00C1100203B600F71230F5128BC875440327
:1031CD00124A1E12A7DAD54403022FC0201EF17831
:1031DD009F7680754A0012B424D210754E50C211DC
:1031ED00C213C212124997C24675A60A12BC852097
:1031FD001203123785E5A624FA40061249E775A693
:10320D000A20251FE59054067008E53524E2501676
:10321D008011E54375F00AA4242295355008E590F8
:10322D0020E2030232BC201E1DE53224104017207F
:10323D0046142428500D30410AE537B40205129288
:10324D00CDD2461239E1D2AC306DAA12D223B4E000
:10325D00A4124A64302B187F572012027F5675A78F
:10326D00009004DFE0A24A92E7C24AF012355E30C8
:10327D004108E537B402031292CD1233B91239E188
:10328D00129FD912B80C1239E1128BC830121D12CF
:10329D00B7F812B4CBE5510404F57F24FE40037555
:1032AD007F02C277E54024EF5002D2550231F13052
:1032BD002B057F5812355E75A6FFC210301208D24D
:1032CD0021124A421232DCC212752F00020136124F
:1032DD00B66A12D4C3E47E057F1E909C0312731848
:1032ED0012D30F12D3DDD214D2201216E1852BBCCE
:0932FD008521BD75B90575B90202
:1033060012B674D25512B56A7F0012B4B1D2201229
:10331600B674E56A600512B52E80F7857A62D2200A
:103326001216FF85BEBC85BFBD856BBE856CBF759D
:10333600B90575B90285BD6C85BC6B756A2012B678
:103346006A1235F912B5A912B674756A0012B61169
:10335600E57064FE70437570FC854077854178851D
:103366001F797818797A12BFE512B5137FB412B5B2
:1033760095D22012D3EB12B674756A1012B6118567
:1033860054717F087810797212BFE785627C855E7A
:103396007D12B5137FC412B595302B1230210F1252
:1033A600358D30430912CC0412D30F12D3DAC22062
:1033B600C21422300A01221249B412350A7452127A
:1033C600D073744D12D073744312D0731235191220
:1033D600D0AE7441207402745612D0731234661241
:1033E60034B012D0AEE53C12D066E53B12D066E5AD
:1033F6003A12D0661234E612D0AE744512D0731269
:10340600354F12350A744712D073744712D073744D
:103416004112D07312351912346612D0AEE43074EC
:10342600010412D07112D0AE9004C3E012D066121D
:10343600D0AE9004E4E075F00A84AFF012D06612C4
:10344600D0B2EF12D071AC5EAB7A12352BAC5DAB5D
:103456005C12352B12D0AE12D0AE12354F02499700
:103466007875C23D1234717878D23D12D0AE127D95
:10347600EC303D05E51E12D071E51D12D0711234F7
:06348600F3E51812D071FD
:10348C00E57D203D01C4540F12D07112D0AE303DF9
:10349C0009744530170274578007744E3017027444
:1034AC005302D0732074081234E61234E680277568
:1034BC00A7049004BFE0FCE0FB7A1B12648B78320B
:1034CC0012662D1264531234F09004C1E0FCE0FB40
:1034DC001264531234F075A7002212D0AEE4F51A20
:1034EC00F519800D12D0AEE51C12D071E51B12D06F
:1034FC0071E51A12D07112D0B2E51902D071742490
:10350C0012D073744712D0D8745002D07312D0AE4C
:10351C00E53D12D066E53E12D066E53F02D066125C
:10352C007E4812D0AEE51D12D073781CE612D07115
:10353C0018B817F812D0B2E412D07112D0AE744D84
:10354C0002D073C038742A12D073D03812D08D02C6
:10355C00D3EB7D031249C1753800744012D07FEF54
:10356C0012D07F7E3275A7049004B4E012D07FDEB7
:10357C00FAE53812D07F7E011235DB5047DDD5805D
:10358C00437D031249C1753800744012D07F745AC0
:10359C0012D07F7E2075A7049004B4E012D07FDE99
:1035AC00FA75A7007EF0744112D07FDEF97EF074BC
:1035BC004212D07FDEF9E53812D07F7E231235DB44
:1035CC005002DDBF924375A70012D3EB024997302E
:1035DC0099FD1249C1D2AC12D223C5F07004DEF7AA
:0435EC008007C5F09F
:1035F000B451028001D3C2AC2278107F0EE4F608E9
:10360000DFFCF564F565F567F5687515FC751AC09E
:10361000751DC0756640756940754A0112B5B730B1
:1036200055030236B512B52EE571B510004002F50E
:1036300010E57EB511004002F511E512207502E596
:1036400013C395795006207545857913D3E57A958E
:1036500014E5156480FFE55E64809F400C857A1454
:10366000855E15857B16855F173074ADC2D1786491
:10367000797312369378677976123693D2D17818A7
:103680007973123693781B7976123693808B85790D
:103690001280B9D3E7960809E7960809E66480FF27
:1036A000E764809F20D101B3400AE7F61819E7F6D6
:1036B0001819E7F622E51AB4C00E7873791812BF0C
:1036C000E57873796412BFE578187964C2D112374E
:1036D0002674181267DE8E47AE1EAF1F781B7967FF
:1036E000D2D1123726C3E51F9FE51E9E50048E1EC1
:1036F0008F1F7EFF7FFFAC1EAD1F1265967A04EF11
:103700008AF0A4E5F0CE8AF0A42EFEE435F0BEFFE8
:02371000011E98
:1037120060051460057EFF8E1F22EE7E0020E7F713
:103722007EFE80F3C3E697FB0809E697FC0809E6EC
:1037320097FD1818191930E703126718C3EB33FB0A
:10374200EC33FCED33FDEB33EC33FBED33FC30D1EA
:1037520005AA471264B40BBB00010C751E03751F4A
:10376200FFEC24FC40048C1E8B1FE627FB0809E6B5
:1037720037FC0809E637A2E713F618EC13F618EB44
:1037820013F62210131978B5E624FA4012E57124D3
:10379200F64008E57924F64002802E0606802AD2F9
:1037A20020753612D22EE4F534F537F55A12B6C525
:1037B2001237D1C219D236C2571295FE12962B85F4
:1037C2003F4DD212205E02D228123169C22022D28B
:1037D20014123821E6F008DFFB857A621238177579
:1037E20070FE783A797112BFE512B5131238178557
:1037F200627A855E7B1216F585BC7E85BD7F75700B
:10380200C012B513123821E0F608DFFB75A7007568
:023812007F0134
:10381400C2142274FF7870F608B880FB2275A704DE
:103824009004F078707F102212232D12BFCC12B7AF
:10383400DE9004EAECF09004EBEBF012498A751F79
:10384400031227B57F6412D3EDD51FF51230F5129C
:10385400D4C312D30FC25AC258C259756A2012B5C2
:10386400B71267DC8E47754A01753901C210D2114F
:10387400D214D236D21212B6C51295FE12962B75F8
:10388400A6FF753609753200E59054067008E535D3
:1038940024E2502E8011E54375F00BA424199535CC
:1038A4005020E59020E21BC211C21212D4C312D3DD
:1038B4000FE4F535F52FC22D7E0612D3E7C20202BE
:1038C4002432E54A20E01612B7C412498A12D0A560
:1038D400744912D0D8780412D04B12D08DC221B4BE
:1038E4000202D22112B5B7129FD9302611126B6988
:1038F400128BCB753606E53670FCC2268081128B9E
:10390400C81239E1E54A20E021B40209753900E51D
:103914003670F980E7E53960E3FD24E240020539B9
:1039240012B5B72026C7DDF880D275390012498A4E
:10393400D2ACE536602712D21EB440F612D21EB4C1
:10394400400312D21EB44915F53812D24EFC12D2DD
:103954004EFBAD3812D24E6D7003123965C2AC8085
:0C3964009BC39004E9E0FF9B9004E8E0A6
:10397000FE9C50048E048F038C148B137A101264F7
:103980008B74202BF56A9004E7E03CF56B9004E61D
:10399000E03D540FF56C754A0112B5B7AE14AF1384
:1039A0007C0E7D101265968F40AE04AF057C007DC5
:1039B0003C1265968F418D429004EBE02513FF90F9
:1039C00004EAE03514FE7C0E7D1012659678AEA6F2
:1039D00007AE04AF057C007D3C1265968F3E8D3F9F
:1039E0002210002910010D10020D20783020790AD4
:1039F000207A1722023B3D023A9DE53760061460AB
:103A000006023BA7023B51023B8F023AC1E5372435
:103A1000FD500A24FD4003023C23023BF1201147E4
:103A2000753400201203D2132278A9E67010760AAA
:103A3000D277D24AD226753614D22E02B6BA200BCD
:103A400025204122E537B4021DE6B4050B1295FE90
:103A500012962B75360A8009B4080B1295FE75363E
:103A60000578A916D22E2210780122753900E53486
:103A700024384007754A0175340022700AE54A303F
:103A8000E0F2754A0280F0146008754A0612962B1F
:103A90008006754A041295FE75390180DA302909CD
:103AA000C229D22A7559008005302A0CD229128DDC
:103AB00094128D6275340022206847302703D26A41
:103AC00022D222123DBC107A0122C249E5342438A8
:103AD0004007753700753400227009E4C53770F56A
:103AE000053780F1C241F5371470040537D24130F3
:103AF0005E0B24FB500E753706D22880D87537022E
:103B000080F78033E537640260CBC228E53724FDB7
:103B10002324BEF879C4E7F9A74809A75979C4E86E
:103B2000F78648088607E537B40405754818D24972
:103B30001230048F59809E123D98023D42E5376055
:103B40001014604B14606024FC4003023C9A023C59
:103B500070D2231243F010790122E5342438400753
:103B600075460175340022700EE54624FE40F1E5ED
:103B70004660ED154680ECB40600500C04F5462472
:103B8000FA50E075460580DB100FD8D20F80D410B4
:103B9000790122E53424374007105B25D25B802170
:103BA00010081ED208801A10790122204135D22E29
:103BB000D24BE5342437400D753603C25AC258C281
:103BC0005975340022D25A7009753609D258C25933
:103BD00080EF75360CC258D2591460E575360FD295
:103BE0005880DE78B8A65E08A67A753605D22E8093
:073BF000D030122B128DCE24
